:10000300C9E420C6B520BFA820BDC920B7D120CFE1
:10001300B520CDB300CEB0C7B6BFC6BCBC00BFA829
:10002300BAC500D3E0B6EE00B6C1BFA8CAA7B0DC1C
:10003300A3ACC7EBD6D8CBA20020202020202020C1
:1000430020202020202020202000C7EBD6D8B3F585
:10005300CABCBBAF0020202020202020202020204D
:100063000025302E31660041433741334537340094
:10007300D4AA000313010A210004FFFFFFFFFFFFBF
:100083000A210006FFFFFFFFFFFF0E230005FFFF0E
:10009300FFFFFFFF523020100A240005FFFFFFFF80
:1000A300FFFF0E250005FFFFFFFFFFFF020000001B
:1000B3000E260005FFFFFFFFFFFF020000000212F4
:1000C3001A943357335722F612732B161AB50A3381
:1000D3001A9422D6127422D622F622B522D51A9465
:1000E30012941AD512B51AD612B50A9502540213F0
:1000F300023402340234023402340254025402340D
:100103000234023402340254025502550255025598
:1001130002550255025502350235023502350235C4
:100123000235023502350235023502350235023514
:100133000235023502350235023502350235023504
:1001430002350235023502350235023502350235F4
:1001530002350235023502350235023502350235E4
:1001630002350235023502350235023502350235D4
:1001730002350235023502350235023502350235C4
:1001830002550255025502550255025502550255B4
:1001930002550255025502550255025502550255A4
:1001A3000255025502550255025502550255025594
:1001B3000255025502550255025502550255025584
:1001C3000255025502550255025502550255025574
:1001D3000255025502550255025502550255025564
:1001E3000255025502550255025502550255025554
:1001F3000255025502550255025502550255025544
:10020300025602560256025602560256025602562B
:10021300025602560256025602560256025602561B
:10022300025602560256025602560256025602560B
:1002330002560256025602560256025602560256FB
:1002430002560256027602760276027602760A9504
:1002530002525CD9E7DFE79EEF9FDF3EC6BEC6DFF3
:10026300DF1FDF3FDF5EE75FE77FEF7FEF9FEF9FFC
:10027300EF9FEF9FEF9FEF9FEF9FEF9FEF9FF79F03
:10028300EF9FEF7FEF7FEF7FE77FE77FDF7FDF5F2B
:10029300D73FCF1FC6FEC6DEBEBFBEBFB6BFB69F2B
:1002A3001273125312532B37337812742B372B5884
:1002B3001AB51A9522F61254127422F622D51AB5DB
:1002C30022F612B51AF612B512B51AF612B612952F
:1002D30002750234025502350235025502550235C4
:1002E3000255025502550255025502550255025553
:1002F3000255025502550255025502550255025543
:1003030002550255025502350235023502350235D2
:100313000235023502350235023502350235023522
:10032300023502350236023602360236023602360C
:1003330002360236023602360236023602360236FA
:1003430002360236023602360236023602360236EA
:1003530002360236023602360236023602360236DA
:1003630002560256025602560256025602560256CA
:1003730002560256025602560256025602560255BB
:1003830002550255025502550255025502560256B0
:10039300025602560256025602560256025602569A
:1003A300025602560256025602560256025602568A
:1003B300025602560256025602560256027602763A
:1003C30002760276027602760276025602560256CA
:1003D300025602560256025602560256025602565A
:1003E300025602760276027602760276027602766A
:1003F300027602760276027602760276027602763A
:100403000276027602760276027602760276027629
:100413000276027602760276027602760276027619
:1004230002760276027602760297029702960232EB
:100433003374AEFEE79FE79FD75FBEDEB6BEC6DF6F
:10044300D73FDF3EDF3FE75FE77FE77FEF7FEF9F4A
:10045300EF9FEF9FEF9EEF9FEF9FEF7FEF7FEF7F8A
:10046300EF7FEF7FEF5FE75FE75FDF5FD73FD71F89
:10047300C6DEBEDEBEBEB6BEAE7EAE7EAE7FAE7F97
:100483003B973B9722F5123312531AB50A330A33BB
:1004930022F6335822D62B172B1712741A941AB537
:1004A30012741AD5231622F622F61AB51AD61AD6BC
:1004B3001295023402330234023402340234023419
:1004C3000234023402340234023402340234023479
:1004D3000234023402540254023502350235023426
:1004E3000234023402340234023402340234023459
:1004F3000234023402340234023402340234023449
:100503000234023402350235023502350235023532
:100513000235023502350235023502350235023520
:100523000235023502350235023502350235023510
:100533000235023502350235023502350235023500
:1005430002550255025502550255025502550255F0
:1005530002550255025502550255025502550255E0
:1005630002550255025502550255025502550255D0
:100573000255025502550235023502350255025520
:1005830002550255025502550255025502550255B0
:1005930002550255025502550255025502550255A0
:1005A300025502550255025502550255025602568E
:1005B3000256025602560256025602560256025678
:1005C3000256025602560256025602560256025668
:1005D300025602560256025602550255025502555C
:1005E300025502550255025502560256025602762C
:1005F300027602550255027602760276027602767A
:1006030002760276027502950276027702351AD4D3
:100613008DFCC73ED75EDF7FCF1FBE9DBEBDC6FE2E
:10062300CF1ED73FDF3EE75FE75FE77FE77FEF7FE1
:10063300EF7FE79FEF9EE79FE79FE77FE77FE75F18
:10064300E75FE75EDF3EDF3FD71FCEFFC6DEBEBEFE
:10065300B69FAE7EAE5EAE5EA63EA65EA65EAE5E06
:1006630043964BF7649A64BB5C7A649A64BA5459B0
:1006730043B643B643D743D74C185C5A5C7B5C7A8A
:10068300545A54194BD85439541954594C184C389A
:100693004C184C194C193BD73BB83B973B973BB88D
:1006A3003BB83BB833B83BB83BB83BB83BB83BB8B7
:1006B3003BB83BB83BB83BB83BB83BB83BB83BB89F
:1006C3003BB83BB83BB83BB83BB83BB83BB83BB88F
:1006D3003BB83BB83BB83BB83BB83BB83BB83BB87F
:1006E3003BB83BB83BB83BB83BB83BB83BB83BB86F
:1006F3003BB83BB83BB83BB83BB83BB83BB83BB85F
:100703003BB83BB83BB83BB83BB83BB83BB83BB84E
:100713003BD83BD83BD83BD83BD83BD83BD83BD83E
:100723003BB83BB83BB83BB83BB83BB83BB83BB82E
:100733003BB83BB83BB83BD83BD83BD83BD83BB89E
:100743003BB83BB83BB83BB83BB83BB83BB83BB80E
:100753003BB83BB83BB83BD83BD83BD83BD83BB87E
:100763003BD83BD83BD83BD83BD83BD83BB83BB82E
:100773003BB83BB83BB83BD83BB83BB83BB83BB8BE
:100783003BB83BB83BB83BB83BB83BD83BD83BD86E
:100793003BD83BD83BD83BD83BD83BD83BD83BD8BE
:1007A3003BD83BD83BD83BD83BD833D83BD83BD8B6
:1007B3003BD83BD83BD83BD83BD83BD83BD83BD89E
:1007C3003BD83BD83BF83BF833D93BF93BF93BF9F2
:1007D3003BF93BD933D83BF93BF93BF93BF93BD9DF
:1007E3003BF93BF93BD93BF93BD83BD76CFA9E1C11
:1007F300DF9FDF3EDF5EDF5FD73FCF1FCF1FCF1F00
:10080300CF1FD73FDF5FE77FE77FE77FE77FEF7F9D
:10081300EF9FE79FE79FE79FE79FE77FE75FE75F3D
:10082300DF3FDF5FD73FD71FCF1FC6FFC6DFBEBF88
:10083300BEBFB69FB69FB69EB69EB69FB69FB6BFC7
:1008430074FA6478541754166CB95C78541764B905
:10085300751B74FA64B9751B6CDA5C585C186459BF
:100863005C38649974DB6CBA6C99649964796479C3
:100873005C5864996479649A649A5C79543954181D
:1008830054195419541954195419541954195419FD
:10089300541954194C1954195419541954195419F5
:1008A30054195419541954195419541954195419DD
:1008B30054195419541954195419541954195419CD
:1008C300541954194C384C384C384C384C384C3833
:1008D3004C384C384C394C394C394C394C394C39EF
:1008E3004C394C394C394C394C394C394C394C39DD
:1008F300543954395439543954395439543954398D
:1009030054394C3954395439543954395439543984
:100913004C394C394C394C3954394C394C394C39A4
:100923004C394C394C395439543954395439543974
:1009330054394C3954395439543954395439543954
:10094300543954395439543954395439543954393C
:100953005439543954395439543954394C394C393C
:100963004C394C394C394C394C394C394C394C395C
:100973004C394C394C394C394C394C394C394C394C
:100983004C394C394C394C394C394C394C394C591C
:100993004C394C394C594C594C5A4C594C5A4C5A69
:1009A3004C594C5A547A4C7A4C7A547A4C594C5987
:1009B300545A54595459543A4C3A4C3A4C3A4C5A66
:1009C300545A545A4C5B4C5A545785BAD7DFDFBF3D
:1009D300E77FEF5FE75EDF3ED73FCF1FCF1FC6FF47
:1009E300CEDFCEFFD73FD75FDF5FDF5FDF5FDF5F46
:1009F300DF5FDF5FDF5FDF5FDF3FD73FD71FD71FDC
:100A0300D71FCF1FC6FFC6DFBEDFBEBFB6BFB69EB2
:100A1300B69EB69EB69EB69EB67EB69EB69EB6BF32
:100A230074FA7D5C7D3B74D95C165C586CDB5C3876
:100A330053F75C5864995417647974FB74DA6CBA8D
:100A430074DA6C995C3864585C3864586C9A6479CD
:100A53006479647A647A649A64595C595C59541968
:100A630053F84BF954194BF94BF94BF94BF94BF933
:100A73004BF94BF94BF94BF94BF94BF94BF94BF953
:100A83004BF94BF94BF94BF94BF94BF94BF94BF943
:100A93004BF94BF94BF953F953F953F94BF94BF91B
:100AA3004BF94BF94BF94BF94BF94BF94BF94BF923
:100AB3004BF94BF94C194C194C194C194C194C194D
:100AC3004C194C194C194C194C194C194C194C19FB
:100AD3004C194C194C194C194C194C194C194C19EB
:100AE3004C194C194C194C194C194C194C194C19DB
:100AF3004C194C194C194C194C194C194C194C19CB
:100B03004C194C194C194C194C194C194C194C19BA
:100B13004C194C195419541954195419541954197A
:100B2300541954195419541954195419541954195A
:100B3300541954195419541954194C394C394C3902
:100B43004C394C394C394C394C394C194C1A4C1AD8
:100B53004C1A4C1A4C1A4C1A4C1A4C1A4C1A4C1A62
:100B63004C1A4C1A4C1A4C1A4C1A4C1A4C1A4C3A32
:100B73004C3A4C1A4C1A4C3A4C3A4C5A4C5A4C5A22
:100B83004C5B4C5A4C5B549B4C9B4C7A4C5A4C5A86
:100B9300545A4C3A543A4C1A4C1A4C1A4C1A4C1A92
:100BA3004C1A541A4C3A4C59753ABF3FD77EDF5E04
:100BB300E77FE75FDF3ED71ECF1FC6FFBEBFB6BFCF
:100BC300B69EB69EBEBFBEDFBEDFBEDFBEDEBEBE0E
:100BD300BEBEBEDEBEDEBEBEBEBEBEBEBEBEBE9E12
:100BE300B69EB69EAE7EAE7EAE7EAE5EA65EA63EE2
:100BF300A63EA63EA63EA63EA63EA63EA65EAE5E8A
:100C030053F753F76C99751B7D5C751B6CDA753B59
:100C1300753C647954386CDA649954385C7964B9F6
:100C2300543864996CFA6CDA6CDA6CBA5C595C59B6
:100C33005C795C59649A5C7A64B96CDA5C795C7946
:100C43005C7A54394BF94BF94C184C194C194C1923
:100C53004C194C194C194C194C194C194C194C1969
:100C63004C194C194C194C194C194C194C194C1959
:100C73004C194C194C194C194C194C194C194C1949
:100C83004C194C194C194C194C194C194C194C1939
:100C93004C194C194C194C194C194C194C194C1929
:100CA3004C194C194C194C194C194C194C194C1919
:100CB3004C194C194C194C194C194C194C194C1909
:100CC3004C194C194C194C194C194C194C194C19F9
:100CD3004C194C194C194C194C194C194C194C19E9
:100CE3004C194C194C194C194C194C194C194C19D9
:100CF3004C194C194C194C394C394C394C194C1969
:100D03004C3A543A4C394C194C194C394C394C39EE
:100D13004C394C394C394C394C394C394C394C39A8
:100D23004C394C394C394C394C394C3A4C3A4C3A95
:100D33004C3A4C3A4C3A4C3A4C3A4C3A4C3A4C3A80
:100D43004C3A4C3A4C3A4C3A4C3A4C3A547B4C7AE7
:100D53004C5A4C5A4C5A549B54BB54BB4C9B4C9BC3
:100D63004C9B4C9B54BB4CBB4CBB4C9B4C9B4C7B00
:100D73004C5A545A4C3A4C3A4C3A4C5A545A547A68
:100D8300547B547B5CBA965EC75FD77FEFBFF7DFB8
:100D9300EFDFEFFFEFFFE7BFD77FC73FBEFFB6DF52
:100DA300B6BFB6DFB6DFB6DFB6DFB6DFB6DFB6BFD8
:100DB300B6BFB6DFB6DFB6DFB6DFB6BFB6BFB6BF08
:100DC300AEBFAE9FAE9FAE9FAE9FAE9FAE7FAE7FD8
:100DD300A67FA65FA65FA65FA65F9E1E961E9E1EAB
:100DE3007D1B6CDA5C1753F66458649A54185418D4
:100DF300649A751C753C64BA6CDB751B6CBA6479B8
:100E03006CDA649A54185C795C585C5864BA6CDB8D
:100E1300649A6CDA64BA64BA64995C795C795C79D3
:100E23005C9A5C7A5C9A5C9A54384C184C184C194E
:100E33004C194C194C194C194C394C394C394C3907
:100E43004C394C184C184C194C194C194C394C3919
:100E53004C394C394C394C394C394C394C394C3967
:100E63004C394C394C394C394C394C394C394C3957
:100E73004C394C394C3A4C3A4C194C394C3A4C3A63
:100E83004C3A4C3A4C3A4C3A4C3A4C194C3A4C3A50
:100E93004C394C394C394C394C394C394C394C3927
:100EA3004C394C394C394C394C394C394C394C3917
:100EB3004C394C394C394C394C394C394C394C3A06
:100EC3004C3A4C3A4C394C394C394C394C394C3AF4
:100ED3004C3A4C5A4C5A4C5A4C5A4C5A4C3A4C3A3F
:100EE3004C3A4C3A4C3A545B545B4C3A4C5A4C5A3D
:100EF3004C5A4C3A4C3A4C3A4C3A4C3A4C3A4C3A9F
:100F03004C3A4C3A4C3A4C3A4C5A4C5A4C5A4C5A2E
:100F13004C5A4C594C594C594C594C594C594C59A5
:100F23004C594C594C794C794C9A4C9A54DB4CBBE8
:100F33004CBB4CBB4CBB54DB4CDB4CDB4CDB4CBBEE
:100F43004C9A4C9B4CBB4CBB4C9B4C9B447B4C5B8F
:100F53004C5B4C7B4C7A4C794C583BB62B1322D2CE
:100F630022B21AB222F243B54BF554165C355C1427
:100F73005C145C135C1453F44BD443944395439433
:100F83004374439543953B943B94439443944394D4
:100F930043943B9443944394439543743B743B740D
:100FA3003B743B943B943B943B943B743B743B5466
:100FB3003B543B553B753B753B336CD9961D95DDD7
:100FC3007D3B857B857C7D3B64795C387D3C751CF2
:100FD3005C3853F75C1864795C185C176C99751B63
:100FE300649964BA751C64BA64BB6CFB649A5C59FB
:100FF3005C595C79649A64BA647A6CFB6CFB649A9E
:101003005C79649A649A5C79647A5C5A4BF85419F3
:101013004C1A4C1A4C1A4C1A4C3A4C3A4C394C3A1E
:101023004C394C394C394C194C194C194C394C39F5
:101033004C394C394C394C394C394C394C394C3985
:101043004C394C394C394C394C394C394C194C19B5
:101053004C394C394C194C194C194C194C194C1925
:101063004C194C194C194C394C3944194C194C191D
:101073004C394C394C394C194C194C194C194C19E5
:101083004C194C194C194C194C194C194C194C1935
:101093004C194C194C194C194C194C194C194C1925
:1010A3004C194C194C184BF84C184C194C184C183B
:1010B3004C184C394C394C394C394C184C184BF8AA
:1010C3004C184C184C184C184C184C184BF94BF93D
:1010D3004BF94BF94BF94BF94BF94BF94BF94BF9ED
:1010E3004BF94BF94BF94BF94BF94BF94BFA4BFADB
:1010F3004BFA4BFA4BFA4BFA4BFA43FA43FA43FADD
:1011030043FA441A441A441A443A445B447B447CE9
:10111300447C447C4C9D449D3CBC44DC44DC44BC4A
:1011230044BC44DC449C4C5B4C3A4C3A4C3A4C1A1D
:101133004C1A4C1A4C3A443A443A441A43D93B9811
:1011430033982B561AF612F60AD602D602B702B70E
:1011530002F802D802D702D702D702F702D702D782
:1011630002D602D602D702D702D702D702F702F776
:1011730002F703170338033703170317031703177C
:10118300031802F802D702B7029702970297027672
:1011930002950295029502B502534C7A961E8DBCB8
:1011A3004BF654176499751B859D857D74BA74DA63
:1011B300855C853C6C996C99855C74DA5C58541732
:1011C3005C585C79543864BA64BA64996CDB751CF6
:1011D3006CFB6CDB6CDB649A64BA649A5C79649A2A
:1011E300649A649A649A6CDB64BB649A649A545AF2
:1011F3004C194C194C1A4C3A4C3A4C394C394C3921
:101203004C394C394C394C394C394C394C394C39B3
:101213004C394C394C394C394C394C394C394C39A3
:101223004C394C394C394C394C394C394C3A4C5A71
:101233004C5A4C5A5459545A545A547A547A547AEC
:10124300547A547A547A549A547A547A547A549AEB
:101253005C9A5C9A5C9A5C9A5C9A5C9A5C9A5C9ADB
:101263005C9A5CBB5CBB5CBB64BB64BB64BB64BBC4
:1012730064DB64DB64DB64BB64BB64DB64DB64DAB4
:1012830064DA64DA64FB64DA64FA6CFB6CFB6CFAB0
:101293006CFA6CFA6CFA751A751A6D1A6D1A6D1A66
:1012A3006D1A751A751A751A751A751A751A751ACB
:1012B300751A753A7D3A7D3A7D3A7D3A7D5A7D3A83
:1012C3007D3A7D5A7D5A7D5A7D5A855A855A855A6B
:1012D300855A857A857A857A855A8D5A8D5A8D5A9B
:1012E3008D5A855A857A857A857A859B859B859BD8
:1012F300859B85BB85BC85DC85DC85DC85DC85DC65
:1013030085DC85BC7D7B7D7B7D7B7D7A7D5A7D5AAB
:10131300753A753A753A753B753B753B755C755C0B
:10132300755C757C6D7C7E1E867F6DFD5D9C2C9B44
:101333000BBA03DC0BBC03BD03FF03FF03FF03DE98
:1013430003DD03FD041E041E043F043E045F0C7F03
:10135300047F049F04BF049F045F045F043F041ED3
:1013630003FE03DE03DE03BD03BD03BD03BD039D17
:10137300039D03BD03BD0BBC0B5954FC965F95FE47
:101383007D5C6CDA5C3853F75438649A649A4BF793
:101393005418649A7D5C7D3C5C7974FB857C7D3C50
:1013A300751B753C753C64BA5C5964BA5C795C79AD
:1013B3005C795C595C796CDB6CBA64BA74FB751C40
:1013C3006CDB649A64BA649A5C595C7A64BB5C9B18
:1013D30064BB5C9B54394C394C394C3A4C394C3ACC
:1013E3004C394C3A4C3A4C3A4C3A4C3A4C3A4C3ACB
:1013F3004C3A4C3A4C3A4C3A4C3A4C3A4C3A4C3ABA
:101403004C3A4C3A4C3A4C3A4C3A4C3A4C3A4C3AA9
:101413004C5A4C5A4C5A545A545A545A545A545A71
:10142300545A547A547A547A547A547A547A547A69
:10143300547A5C7A5C7A5C9A549A549A5CBA5CBB30
:101443005CBB5CDB5CBB5CDB64DB64BB64BB5CBB69
:101453005CBB5CBB5CBB5CBB64BB64BB64DB64DB71
:1014630064DA64DA64DA64DA64FB6D1B6D1B6D1B8A
:1014730064FB64FB64FB64FB64FB64FB64DB6CDBA9
:101483006CDB6CDB6CFB6CFB6CFB6CFB6CFB6CFB61
:101493006D1C753C753C751C6D1B6D1B6D1B6D1BAD
:1014A3006D1B751B753B753B753B753B753B753B01
:1014B300753B755B755B755B755A755B755B757BAA
:1014C300757B757B757B757B6D7B6D9B6DBB6DBB19
:1014D3006DDC75FC761D761D7E1D7DFD75BC759CD2
:1014E300757C6D3B755B6D3C6D3C6D3C6D3C6D3C43
:1014F3006D3C6D3C6D3C653B653B6D3B653B653BC6
:10150300655B65BC7DFD8E3E967D9E9DA6BE967FEA
:10151300759D54DC2BFA1379035A037B039D03BD9A
:1015230003BC03FD043D043D045D047E047E049E70
:10153300049E045E0C5E043D0C1D0BFD03DC0BBC22
:1015430003BC03DC03DC03BC03BC03BC03BC03BC60
:1015530003BE03BE03BE03BD0B3954DC9E3F9DDDBA
:101563007D3C8D9E8DBE7D5C6C99541764BA7D7DE8
:1015730064BA54584BF75C59649A5C3854176499AD
:10158300753B5C595C796D1B755D751C6CFB753C1B
:101593006CDB751C6CDB5C795C59649A6479649AC6
:1015A300649A64BA64BA649A6CFB64BB649A64DB3D
:1015B30064BB5C9A5CBB54594C394C394C394C3A3A
:1015C3004C3A4C3A4C3A4C3A4C3A4C3A4C3A4C3AE8
:1015D3004C3A4C3A4C3A4C3A4C3A4C3A4C3A4C3AD8
:1015E3004C3A4C3A4C3A4C3A4C3A4C3A4C3A4C3AC8
:1015F3004C3A4C3A4C3A4C3A4C3A4C3A4C3A4C3AB8
:101603004C3A4C3A4C3A4C3A4C3A4C3A4C3A4C3AA7
:101613004C3A4C394C394C39443944594C7A4C9AEC
:101623004C9A4C9A4C7A4C7A4C5A4C5A4C394C1929
:101633004C394C394C394C3A4C3A4C394C394C397D
:101643004C394C594C594C394C394C594C5A4C7BAC
:101653004C5A4C3A443A443A443A443A4C1A4C1A97
:101663004C1A4C1A4C1A4C1A4C1A4C194C394C390A
:101673004C394C39443944394C394C39441944199F
:1016830044194C394C394C394C39441A441A441ACC
:10169300441A441A441A441A441B4C1B4C1B441B43
:1016A300441B441B443B443B4C7C4C9C4CBC4CDD9A
:1016B3004CFE4D1E4D3F4D5F4D5E4D1D44DD44BC04
:1016C300447B445B445B445A445A445A445A445A04
:1016D300445A445A4C5A4C3A4C3A4C5B4C3A4C5A46
:1016E3004C9B54FD5D7E65BE659D6D7C759C7D9DAB
:1016F30085BD8DDE7DDF6D9E449C2C1B0B9A039C68
:1017030003FE043F043E0C5F045F045F047F047F19
:10171300045E045E043E041E03FE03FD03FD03DDBD
:1017230003DD03BD03BD03BD03BD039D039D039DF6
:1017330003BD03BD03DE03BD03594CDC95FE8D9C45
:1017430053F75C3864997D5C8DDD859D751B74FA58
:10175300859D859D7D5C6C9974FA859D753B5C794F
:10176300543764DA6CFB4C185C7964795C595C59C6
:101773006CDB6CDB649A6CFB751C751C6CFB6CFB83
:10178300751C64BA64996CDB649A5C7A64BA64BA53
:1017930064DB64DB5CBA64DB5CDB549A547A4C5ADA
:1017A3004C3A4C5B4C5A4C5A4C5A4C5B4C5B4C5B22
:1017B3004C5B4C5B4C3A4C3A4C3A4C3A4C3A4C3AB4
:1017C3004C3A4C3A4C3A4C3A4C3A4C3A4C3A4C3AE6
:1017D3004C3A4C3B4C3B4C3B4C3B4C3B4C5B4C5B8F
:1017E3004C5B4C3B4C3B4C3B4C3B4C3B4C5B4C3B7E
:1017F3004C5B4C5A4C5A4C5A4C9B4CDC54FC4CFCA6
:101803004CDC4CBB4CBC4CBB4C9B4C7B4C5B4C5A9C
:101813004C7B4C7B4C7B4C7B4C7B4C7B4C7B4C9B6D
:101823004C9B4C9B4C9B4C9B4C7B4C7B4C7B4C7BFD
:10183300547B547B4C5A4C5A4C5A4C5A4C7B4C7BE1
:101843004C7B4C7B4C7A4C7A4C7A4C7A4C5A4C7B82
:101853004C7B4C7A4C7A4C7B4C7B4C7B4C5B4C5B8F
:101863004C5B4C7B547B547B547B4C7B4C7B4C7B45
:101873004C7B4C7B4C7B4C7B4C7B4C7B4C7B4C9B0D
:101883004C9B4C9B4CBC54DC54FC54FC551D553DAB
:101893004D5E557E4D9E557E553D4CFC4CBB4C9B41
:1018A3004C9B547B547B4C7B4C7B4C7B4C7B4C7BCD
:1018B3004C7B4C7B4C7B549C549C549C549C54BC00
:1018C3004CBC4CDC4D3D4D3C4D3C4D3C5D5C6D7C1E
:1018D3007DBC8DDD961EA63E95FE8DDE6D9D451D60
:1018E3001C3B043C045E047E049F049F04BF04BFAE
:1018F30004BF047F043E041E043E041E03FD043E95
:101903000C7F0C5F043E041E03FE03FE03FD03FD78
:1019130003DC03DD03FE03FE0BFC451D7DBE7D9C46
:101923006CDA649954174C184C3964FA753A543884
:1019330053F8647A7D3C85BD751A5C787D3C857D62
:10194300859D751B7D3C859D751B64997D5C7D3CE8
:10195300647964796CDA64795C795C7A5C7964DBE8
:1019630064BB649A6CFB6CFB64BB6CFB6CFB64DB5D
:101973006CFC6CDB5C9A5C9B5CBC64DB5CBB5C9A64
:101983004C5A4C3A4C3B4C3A4C3A4C3B4C3A4C3A02
:101993004C3A445A4C3A4C3A4C3A4C3A4C3A4C3AFC
:1019A3004C3A4C3A4C3A4C3A4C3A4C3A4C3A4C3A04
:1019B3004C3A4C3A4C3A4C3A4C3A4C3A4C3A4C3AF4
:1019C3004C3A4C3A4C3A4C3A4C3A4C3A4C3A4C3AE4
:1019D3004C3A445A445A4C9B4CBC54DC54DC4C9B0C
:1019E3004C7A445A447B445B445A445A445A4C5AB2
:1019F3004C5A4C5A4C5A4C5A4C5A4C5A4C5A4C7B93
:101A03004C9B4C7B4C9B4C7B4C7B4C7B4C7B4C7A5C
:101A13004C5A4C5A4C3A4C5A4C5A4C5A4C5A4C5AB3
:101A23004C5A4C5A4C5A4C5A4C5A4C5A4C5A4C5B82
:101A33004C7B4C7B4C5A4C5A4C5A4C5B545B545B1E
:101A4300545B545B545B4C5B4C5B545A4C5A4C5A3E
:101A5300545A4C5A4C5A4C5A4C5A4C7A4C7A4C7AEB
:101A63004C9B4CDB4CFC4CFC4CFC4CFC4CFC4CDCD5
:101A73004CDC4CFC4CFC4CDC549B4C9B4C7B4C7B1F
:101A83004C7B4C7B4C7B4C7B4C7B4C7B4C7B4C7B1B
:101A93004C9B4C9B4C9B4C9B4C9B4CBB44BB44DB9B
:101AA3004CDC4CDC44FD451D4D1B659C75DD85DD23
:101AB3008DDDA65F9E5F95FD95DC9E3DAE9EAEFFE0
:101AC300A6BF5D7C2CBC1CBD1D1E14FF04BE04DF21
:101AD30004BE0C9E0C7D047E047E045E043E0C7EDC
:101AE3000C7E043E03FD03FD03FE041E041D041DC2
:101AF30003FC0C1C043F043F03FD451D861D85BCF0
:101B03008D9D95FE8DBD7D1B647953F754387D5CA7
:101B1300751A649854165C386CBB5C9A4C1754590C
:101B230064BA751C54385C796CFB7D7C64FA64DAA6
:101B3300757C7D9D753B755B753C753C7D5D6CFB74
:101B43006D1C6D1C64BA5C9A6CDB64DB64BA6CFB61
:101B53006CFC6CFB753C6CDB74FB751B751B753C7B
:101B6300753C64BB5C9B5CBC5CBC5CBC5CBC64BB2C
:101B730064BB64BB5CBB5CBC5CBC5CBC5CBC5CDB76
:101B83005CDB5CDB64DB64DB64DB64FB64FB64FB0A
:101B930064FB651B651B651B651B651B651B651B63
:101BA300651B6D1B6D1B6D1B6D1B6D1B6D1B753BD2
:101BB3006D3B6D5B757B757C757B755B755B6D3B99
:101BC3006D3A6D3A6D3A6D3A753A753A753A753BB9
:101BD300753B753B753B753B753B753B753B753B82
:101BE300755B755B755B755B755B755B755B755B72
:101BF300755B753B6D3B753B6D3B753B6D3B6D3B62
:101C03006D3B6D3B6D1B6D1B6D1B6D1B6D3B653B19
:101C1300651B653B651B651B651B651B651B651BA1
:101C2300651B651B651B5D1B5CFB5CDC5CDC5CDCBA
:101C33005CDC5CDC5CDC5CDC5CDC5CDC5CDC5CFCC1
:101C43005CFD5D3D5D5D551D54DC54DC54DC54BCD2
:101C530054BC54BC54BC54BC54BC54BC54BC549C21
:101C6300549C549C549C54BC54BC54BC54BC54BC51
:101C73004CBC4CBC4CBC4CBC4CDC4CFC4CFD4D1D1E
:101C8300553E555E553E5D3C861DAEFFAE9FA63E5E
:101C93009E3E9E5F95FE8DDD95DDA67E9E7E8E1D0E
:101CA300967F969F7E1F659E4D5E453E3D3E3D3F22
:101CB30034FE3D5F2D1F147E0C5E043C0C3C0C3B3C
:101CC300143B1C1B245C245C13FB145E0C7E045E1F
:101CD300045F041F03FF03FE0BBB5D7C9EDF963E88
:101CE3006CB96CFA859D95DE9DFE8D9D7D3C7D3B9B
:101CF3008DDD8DDD85BD6CDB649A7D7D85BE751CB8
:101D03005C595438753C74FC5C7A543A5C7A5C9B3D
:101D1300545A5C9B64BB545A5C7A6D1C64DB64BA92
:101D2300753C6CFB6D1C753C755D751C753C6D1CC1
:101D33006CFB6CFB64DB6CBA6CDA64BA64FB64FB4B
:101D43006CFB6CFB64BB547B547B547B4C5B545BE0
:101D5300545A545A545A4C5A4C5A4C5A545A545A28
:101D6300545A545A547A547A547A547A547A547A40
:101D7300547A547A547954795479547954795479F6
:101D830054795479547954795479547954995C99A0
:101D93005C9A5C995C9A5C79547954795459547976
:101DA300547A5C7A5C7A5C7A5C7A5C7A5C7A5C7A88
:101DB3005C795C795C795C795C795C795C795C7978
:101DC3005499547954795479547954795479549968
:101DD300549954995499549954995499549A549A96
:101DE300549A549A549A549A549A549A54BA54BA40
:101DF30054BA54BA549A549A549A549A549A549A30
:101E0300549A549A549A549A4C9A4C9B4C9B4C9B7C
:101E13004C9B549B549B549B549B549C549C54BC2C
:101E230054BC54DC4CDC4CBC4C9B549B549B549B8B
:101E33004C7B4C7B549B549B4C9B4C9C4C9C4C9C94
:101E43004C9B4C9B4C9B4C9C549C4C9C4CBC4CBC0A
:101E53004CBC4CDC4CDC4CFD4D3D555E557F557EFA
:101E6300553D555D6D9D9E7EC73FD73FCEDFADFE91
:101E73009E1E961D9DFD9E1E961E965F8E3F655C63
:101E8300659D655C759D75DE6DBE657E659E659F12
:101E9300659F3D7E1CDD0C5C24BD4D5E657E85BE6D
:101EA3009E7F96BF9EBF967F863F65BF34FF147E9D
:101EB3000C3E143D1C5C2C5C341975BCA69F9E3EE5
:101EC3005C9A43F84C185C796CFB7D7C8DFD6499BE
:101ED30054196CDC7D5D8DDE8DFD74FB6CDA857DC4
:101EE30095DE8D9D7D3C857D8DDE7D7D6CFB859DA9
:101EF30085BE751B64DA7D5D753C5C9A64BA6D1CA6
:101F0300649A64BA6CFB64BA5C7964BA6CDB5C9AFD
:101F130064BB6CDB64BA6D1C651C651D653D651C8B
:101F230064DA64B96CD954584C174C384C7A4C5C0D
:101F33004C5C4C5B4C5B4C5B4C5B4C5B4C5B4C5B65
:101F43004C5B4C5B4C5B4C5B4C5B4C5B4C5B4C5B56
:101F53004C5B4C5B4C5B4C5B4C5B4C5B4C5B4C5B46
:101F63004C5B447B447B447B447B447B447B447C8D
:101F73004C7B4C7B4C7B4C7B4C7B4C7B4C7B4C7B26
:101F83004C7B4C7B4C7B4C7B4C7B4C7B4C7B4C7B16
:101F93004C7B4C7B4C7B4C7B4C7B4C7B4C5B447B2E
:101FA300447B4C7B4C9B4C9C4C9C4C9C4C9C4CBC19
:101FB3004CBC4CBC4CBC4CBC4CBC4C9C449C449C4E
:101FC300449C449C449C449C449C449C4C9C4C9CFE
:101FD3004C9C4C9C4C9C4C9C4C9C4C9C4C9C4C9CBE
:101FE3004C9C4C9C4C7C4C9C4C7C4C9B4C9B4C9BF1
:101FF3004C9B4C9B4C9B4C9B4C9B4C9C4C9C4C9CA3
:102003004C9C4C9C4C9C4C9C4CBC4CBC4CBC4CBC0D
:102013004CBB4CBB4CBB4C9C4C9C4C9C4C9C4C9C20
:102023004C9C4C9C4C9C4C9C4C9C4C9C4C9C4CDC2D
:102033004CDD54FD54FD4D3D4D3D4D1D4D1C4CDBC4
:102043005CFB7DDDA6BFBEDFC6FED6FFBE5EADFE7A
:10205300A65F9E5F9E3E961E963F7DDE6D9D5D7DD7
:10206300553C4D1C4D1C4CFC4D1C4D1C44FC451C4F
:10207300451C4D5E453E453D65BF75FF9E7FBEFFDA
:10208300BEBEBEBDB69DBEBDB6BE9E7E6D9D557D1C
:102093006DBD7E1E8E9F8E7F8DFE9E5DB69FAE5F55
:1020A3007D7C857D6CFB5C594C194BF85C796D1C10
:1020B30064BB54385418545964DB64DB5458545883
:1020C3005C99753C755C5C795C996D1A85DD6CFA7D
:1020D3005CB9757C85DD755B6CDB859E7D7D753CB0
:1020E3007D7D7D9E7D7E755D755D7D5D753C751C1D
:1020F3006D1C64DB6CFB6D1B5CDA651C64FB649913
:102103009DFBD73DD71DCF1DC6FCB6FD64D94C5AE8
:102113004C7C4C7C4C7B4C7B4C7B4C7B4C7B4C7B82
:102123004C7B4C7B4C7B4C7B4C7B4C7B4C7B4C7B74
:102133004C7B4C5B4C7B4C7B4C7B4C7B4C7B4C7B84
:102143004C7B4C7C4C7C4C7C4C7C4C7C4C7C4C7C4D
:102153004C7C4C7C4C7C4C7C4C7C4C7C4C7C4C7C3C
:102163004C7C4C7C4C7C4C7C4C7C4C7C4C7C4C7C2C
:102173004C7C447C447C447C447C447C447C4C9C2C
:102183004C9C4CBD4CBD4CBD4CBD4CBD4CBD4CBD25
:102193004CBD4CBD4CBC4CBD4C9C4C9C4C9C449C81
:1021A300449C449C4C9C4C9C4C9C4C9C4C9C4C9CFC
:1021B3004C9C4C9C4CBC4CBC4CBC4CBC4CBC4CBC1C
:1021C3004CBC4CBC4CBC4CBC4CBC4C9C4C9C4C9C2C
:1021D3004C9C4C9C4C9C4C9C4C9C4CBC4C9C4C9C9C
:1021E3004C9C4C9C549C549C4CBC4CBC4CBC4CBC1C
:1021F3004CBC4CBC4CBC4CBC4C9C4C9C4C9C4C9C1C
:102203004CBC4CBC4CBC4C9C4CBC4CBC4CBC4CDD8A
:102213004CFD4CFD4CFD4CFD4CFC553C655B7DBCC5
:10222300A67EBEDFC6FFC6FFC71FBEFFAE9FA65F6B
:102233009E5F9E3E8E3E7DDE75DE5D3D4CFC4CDC3E
:102243004CBC44DC44DC44DC44BB44BB553D559EA0
:102253004D5D5D3D759E967F9E7FAE9EB6DFBF3F13
:10226300BEFEB6BEB69EBEDFB6BEA67E9E7F9E9F58
:10227300967F8E7F7E5F761F75FE9E7EBEDFBE7E5F
:102283008D7C9E1E9E1E9E1E8DBD74FB647A74FB08
:10229300963F8DFE7D7C74DB5C3964DB8DFF7D5D59
:1022A3006CDB5C795C797D9E6D1C5C9A545A5C9BFB
:1022B30064FC5C9B547A5CBB5C9A5C7964BA6CFB8F
:1022C3005C9A64BA6D1C5C9A64FC64DB5CBB6D1C39
:1022D30064DB6D1C6D3C6D1B755C6D3C753C74FA69
:1022E300BE7CFFFFFFBEFFFEFFFFEFFF74F75458F6
:1022F300547B4C5C4C7B4C7B4C7B4C7B4C7B4C7BBA
:102303004C7B4C7B4C7B4C7B4C7B4C7B4C7B4C7B92
:102313004C7B4C7B4C7B4C7B4C7B4C7B4C7B4C7B82
:102323004C7B4C7B4C7B4C7B4C7B4C7B4C7B4C7B72
:102333004C7B4C7B4C7B4C7B4C7B4C7B4C7B4C7B62
:102343004C7B4C7C4C7C4C7C4C7C4C7C4C7C4C7C4B
:102353004C9B4C9B4C9C4C9C4C9C4CBC4CBC54DCB4
:1023630054DC54DC54DC4CBC4CBC4CBC54BC54BCA2
:1023730054BC549C549C4C9C4C9C4C9C4C7C4C7C22
:102383004C7C4C7C4C7C4C9C4C9C4C9C4C9C4C9C6A
:102393004C9C4C9C4C9C4C9C4C9C4C9C44BC44BCCA
:1023A30044BC4CBC4CBC4CBC4CBC4CBC4CBC4CBCF2
:1023B3004CBC4CBC4CBC4CBC4CBC4C9C4C9C4C9C3A
:1023C3004C9C4C9C4C9C4C9C4CBC4CBC4CBC4CBC4A
:1023D3004CBC4CBC4CBC4CBC4CBD4CBD4CBD4CBDB6
:1023E3004C9D4CBD4CBD4CBC4CBC4CBC4CBC4CBCC7
:1023F30044BC44BC44BC4CBC5D3D863FA6DFB6FF39
:10240300BEDFC6BFBEBFB69FA69E8E3D7DFD7DDEF1
:1024130075BD75BC6DBD657C54FB4CDB4CBC4CBCC5
:102423004CBC4CBC4CDC4CDC4CFC551C5D7D65BE93
:1024330065BE5D7D4CFA75FD969FA67FB69EBE9EDA
:10244300B6BEAEFFA6DF969F8E7F865F75FF6DBE1D
:10245300559F3D7F2D1E2D1F2CBC7DFCC71FC69D88
:102463006CDA64996CFB857C9DFEA61E9E1E859C82
:102473006CD9859C961E9E3E9E1D7D9C755B8DFD35
:10248300963E8DFD7D9B7D9C8E1E961F859D7D5C5E
:102493008DDE8DDE857D751B859D85BE751C6CDB94
:1024A300859D7D5C6CDB7D5D753C64DB755D6D3CA2
:1024B30064DB6D1C64DB64DA651B5CFC651C5C9788
:1024C300AE5BFFDFF79DF7BDEF9FE7DF74F84C5876
:1024D3004C9C4C7D4C7C4C7C4C7C4C7C4C7C4C7C98
:1024E3004C7C4C7C4C7B4C7B4C7B4C7B4C7B4C7BAF
:1024F3004C7B4C7B4C7B4C7B4C7B4C7B4C7B4C7BA1
:102503004C7B4C7B4C9B4C9B4C9B4C9B4C9B4C9BD0
:102513004C9B4C7B4C7B4C7B4C7B4C7B4C7B4C7B60
:102523004C7B4C7B4C7B4C7B4C9C4C9C4C7C4C9C0C
:102533004C9C4CBC4CBC54DD54DD54FD54FD54FD4B
:1025430054FD54FD54FD54FD54FC54FC54FC551CE3
:10255300551C54FC54FC54DC54DC54DC5CDC5CFC47
:102563005CFC5CFC5CFC5CFC5CFC5CFC64FC64FC98
:1025730064FC64FC64FC64FC64FC651C651D651DF3
:10258300651D651D651D653D653D6D3C6D3C6D3C83
:102593006D3C6D3C6D3C6D3C6D3C6D3C6D3C6D3CF0
:1025A3006D3C6D3C6D3C6D3C6D3C6D3C6D3C6D3CE0
:1025B3006D3C6D3C6D3C6D3C6D5C6D5C6D5C6D5C50
:1025C3006D3C6D5C6D5C6D3C653C653C653C6D5C78
:1025D3006D5C6D5C6D5C6D5D7DBDA69EB6DEBEDE25
:1025E300B6BEB69EAE9EA67E965E85FD75DC6DDCA0
:1025F3006DDD6DBD65DD65DD659D655C655C655C9B
:102603005D5D5D5D653D5D7D5DDD5DBD6DFD75BDE7
:102613007DDE75DE5D9C34B9451B6DBF7DFF7E1E7F
:102623007E1E6DDF557E4D7E3D5E251D14DD0CBD8A
:102633000CBE04BE049E04BF045C75FCD73FD71FC9
:102643006D3C545A4C1954195C5B64BB759D7DBD3C
:1026530054584C37549964FB7DBE7DFE54BA4C5894
:102663005CDA6D5C85FF653C547964DA7D9D85FE9B
:102673006D1B5C9A757D85FF755D5CBA7D9E85DEFD
:102683006D3C755D85BE7D9D6D3C7D9E757D755DE7
:10269300757D757D6D5C7D7D755D757D757C74F86F
:1026A300BEFCFFFFFFFDF7FEF7FFEFFF7CB9545AB7
:1026B3004C7C4C9C4C9B4C7C4C7C4C7C4C7C4C7C98
:1026C3004C7C4C7C4C7C4C7C4C7C4C7C4C7C4C7CC7
:1026D3004C7C4C9B4C9B4C9B4C9B4C9B4C9B4C9BDE
:1026E3004C9B4C9C4C9C4C9C4C9C4C9C4C9C4C9CA8
:1026F3004C9C4C9C4C9C4C9C4C9C4C9C4C9C4C9C97
:102703004C9B4C9B4C9B4C9B4C9B4C9B4C9B4C9B8E
:102713004CBC4CDC4CDC4CDC4CFD4CFD4CFD4CFD12
:102723004CFD4CDC4CDC4CDC4CDD4CDD4CDD4CDD41
:102733004CBC4CBC4CBC4C9C4C9C4C9C4C9B4C9BF8
:102743004C9B4C9B4C9B4C9B4C9B4C9B4CBB4CBB0E
:102753004CBB54BB54BB54BB54BB54BB54BB54BB06
:102763004CBB4CBB54BB54DC54DC54DB54DB54DB5C
:1027730054DB54BB54BB54BB54BB54DB54DB54DB5E
:1027830054DB54DB54DB54DB54DB54DB54DB54DBCE
:1027930054DB54DB54DB54DB54BB54BB54BB54DB1E
:1027A30054DB54DB54DB54BB54BB54BB54BB54DB2E
:1027B30054DB54DB4CDB4D1D555D659D6D9C6DBC41
:1027C30075DD75FE75DE759E655D5D3C553D551D7C
:1027D300551D551D551D54FC54DC54DC54DC54DB91
:1027E30054DB4CDB4CFC551C6D7C7DDD8E1D8DDD7F
:1027F30095FD85BD7DFD869E553A345A453E2D5F38
:102803001D1E14DE0CBD0CBD04BE04BE04DF04DFBC
:1028130004BF04DF04BF04DF045C7E1CE79FDF5FAB
:10282300753B8DDD857C751B5C994C194C195C5986
:1028330085BE7D3C6CBB545A4C1A545A6D1D753D74
:102843005C9B5439543A649B6D3D5CDB4C794C7909
:10285300651C6D3C547A547A5CBB651C549A549A3B
:102863005CDB5CDB547A64FC651C547A5CBB64FC03
:102873005CBA5CDB5CDB5C9B647B64BC64BC649ABD
:102883008D7BB63CADFBADDABE19424818C5112AA3
:102893005439549B4C7A4C7B4C7B4C7B4C7B4C7B10
:1028A3004C7B4C7B4C7B4C7B4C7B4C7B4C7B4C9BCD
:1028B300549B4C9B4C9B4C9B4C9B4C9B4C9B4C9BD5
:1028C3004C9B4C9B4C9B4C9B4C9B4C9B4C9B4C9BCD
:1028D3004C9C4C9C4C9C4C9C4C9C4C7C4C9C4C9CD5
:1028E3004C9C4C9C4C9C4C9C4CBC4CBC4CBC4CBD24
:1028F3004CDD4CFD4CFE4CFD44FD4D1E4D1E4D1E4E
:102903004D1E4CFE4CFE4CFE4CFE4CFE4CFE4CDD74
:102913004CDD4CDD4CDD4CBD4CBD4CBD4CBD4C9D2C
:102923004C9D4C9D4CBD4CBD4CBD4CBD4CBD4CBD9C
:102933004CBD4CBD4CBD4CBD4CBD4CBD4CBD4CDD2C
:102943004CDD4CDD4CDD4CDD4CDD4CDD4CDD4CDD3C
:102953004CDD4CDD4CDD4CDD4CDD4CDE4CDE4CDE29
:102963004CDD4CDD4CDD4CDD4CDE4CDE4CDE4CDE18
:102973004CBD4CBD4CBD4CBD4CBD4CBD4CBD4CBD0C
:102983004CBD4CBD4CBD4CBD4CBD4CBD4CBD4CDDDC
:102993004CDD4CDD4CDD44DE4CFE4D1D4D1D4D3DEF
:1029A3004D3E4D3E4D1E4CFE4CFD44FE44FE4CFE42
:1029B3004CDE4CDE4CFE4CFD44DD4CDC4CFD54FC4B
:1029C30054FC5D3C6DBD8E3EA67FBEBFBEBFC6DF61
:1029D300C6DFBEDEBEFEBF3FB73F75BC245A0CDE6A
:1029E30004FF04FF04FF04FF04FF04DF04DF04BF4C
:1029F30004BF04FF04DF04DF045B863CEFDFDF5E1C
:102A0300857BA65EB6DFB6DFA67D9E3D8DDC857A2F
:102A13009E3DAEBFAEBFA67E9E1D8D9B95FCAEDFD9
:102A2300AEDF9E7E95FC857AA65EAEBFA65E95FC64
:102A33008D9CA63EA67E9E1D8D9C9E3EA65E9E1DE3
:102A430095BC9E1E9E3D95DCA63E9E1D95FD9E3E1D
:102A53009E1D9E1D9E1E8DFD965E8E1E8E1D8E1DC1
:102A63008DBC8DDD857C957D951752A700000001F7
:102A73007CFA6D5D6D5C6D5D6D5D6D5D6D5D6D5D58
:102A83006D5D6D5D653D655D653D653D653D653DC3
:102A9300653C653D651D651D651D651D5D1D5CFD15
:102AA3005CFD5D1D5CFD5CFC5CFC5CFC5CDC5CDC7F
:102AB3005CDC5CBC5CDC5CDC5CBC5CBC54BC54BC03
:102AC30054BC54BC4CBC4CBC54BC4CBC4C9C4CBCCB
:102AD3004CBC4CBC4CBC4CBC4CBC4CBC44DC4CBC9B
:102AE3004CBC4CBC4CBC4CBC4CBC4CBC4CBC44BCAB
:102AF3004CBC4CBC4CBC4CBC4CBC4CBC4C9C4C9CD3
:102B03004C9C4C9C4C7C4C7C4C7C4C7C4C9C4C9C02
:102B13004C9C4C9C4C9C4C9C4C9C4C9C4C9C4C9C72
:102B23004CBD4CBD4C9C4C9C4C9C4C9C4C9C4C9C20
:102B33004C9C4C9C4C9C4C9C4C9C4C9C4C9C4C9C52
:102B43004C9C4C9C4C9C4C9C4C9C4C9C4C9C4C9C42
:102B53004C7C4C7C4C7C4C7C4C7C4C7C4C7C4C7C32
:102B63004C9C4C9C4C7C4C9C4C9C4C9C4C9C4C9C42
:102B73004C9C4C9C4C9C4C9C4C9C4C9C4CBC44BCDA
:102B830044BC4CBC4C9C449C44BC44DC44BC44BC52
:102B93004CBC4CBC44DC4CFD553D5D7D6DBE75DECF
:102BA30085FE963E9E7EBEDFCF1FCEFED71EDF1E66
:102BB300DF3EE75FE73EE75ED71ECF5F75BC13F8E6
:102BC3000CDD04FE04DE04DF04DF04DF04DE04BEE8
:102BD30004DF04FF04DF04DF047C863CEFBFDF5F18
:102BE3008DBD751B7D5C8D9D9E1EAE7EAE9EA69F8C
:102BF300755B6CFA85BC95FDA67EAE9F8DBC64D9D2
:102C03007D7B85FD965EA69F7D5A6D1A85BD963F99
:102C1300965F6D1B6D1B859D963F7D9C6CFA7D9D1C
:102C23008E1E753C64DA7D7D85BE6CFB755C7D7D97
:102C330064DA753C753C64DB753D64DC6D1C6D1CAE
:102C4300651B6D3C653D755C7CF673ED4A4A320D40
:102C5300647A54FD54FC5CDB5CDC5CDC5CFC5CFC9B
:102C63005CFC5CFC5CFC5CFC5CFC5CFC651C651C4F
:102C730064FC64FC64FC64FC64FC64FC64FC64FC51
:102C830064FC64FB64FB64FC651C651C651C64FCE0
:102C9300651B6D1B6D1B6D1B6D1B6D3B6D1B6D1BD9
:102CA3006D1B6D1B6D1B6D1B753B753B6D3B753B49
:102CB300753B753B755B755B755B755B755B6D5BD9
:102CC300755A755A755A757B757B759B759B75BC63
:102CD30075BC759C759C7D9C7D9C7DBC7D9C7D7B22
:102CE3007D7B7D7B7D7B7D9B7D9B7D9B7D9B7D9B81
:102CF3007D9B7DBB7D9B7D9B7D9B7DBB7DBB7D9BB1
:102D03007DBC7DBC7DBC7DBC7DBB7D9B7D9B7D9B5C
:102D13007D9B7D9B7D9B7D9B7D9B7D9B7D9B7D9BF0
:102D23007D9B7D9B7D9B7D9B7D9B7D9B7D9B7D9BE0
:102D33007D9B7D9B7D9B7D9B7D9B7D9B7D9B7D9BD0
:102D43007D7B7D7B7D7B759B759B759B759B757B68
:102D5300757B757B757B7D7B757C757C6D7C6D7CF4
:102D6300757C757C755C757C759C6D9C6D9B6D9C91
:102D730075DD7DFD75DD75BC863E965E9E5DB6BEDA
:102D8300BEBEC6BECEDED71FDF1EDF3EE75EE75EFA
:102D9300EF5FEF9FEF9FEF7EE71EDF1ECF9F6DBAC2
:102DA300143804DE04BE04BF04BF04DF04DF04DF01
:102DB30004FE04FE04DE04BF045B863CEF9FD73FA2
:102DC300961F5C9A4BF94C3A547C64DD6D3D85FE4D
:102DD3007D7D54394C3A4C5A5CFC6D3C759E5CDCF1
:102DE3004C7A4C5A54BC5D1D6D7E54BB4C7A4C7B63
:102DF3005CFC653D54BB4C7A549B5CFC5D1D4C7A7A
:102E03004C9A5CFC653D549A549A6D7D651C549BA9
:102E1300653D6D5D54BB6D3D753D6CDC7D7E755CC4
:102E2300757D759D75BE75DE8D378450ADB995FE84
:102E33005D1E4CDD54DC54DC54DC54DC54DD54DDC9
:102E430054DC54FC5CDD5CDD5CDD5CFD5CFD5CFD49
:102E53005CFD5CFD5CFD5CFD5CFD5CFD5CFD5CFDA7
:102E63005CFD5CFD5D1D651D651D651D651D651DA9
:102E7300651D653D653D653D653D653D653D653D5F
:102E83006D3D6D3C6D3C6D3C6D3C6D5D6D5D6D5D93
:102E93006D7D6D7D6D7D6D9D6D9D759D759D759D27
:102EA30075BD75BD75BD75DD7DDE7DDE7DFE7E1D6B
:102EB3007E1E7E3E863E865E863E863E865E8E5EB7
:102EC3008E5E8E5E8E5E8E5E8E5E963D963D965DCA
:102ED300965D967D965D967D967D967D9E7D9E7D87
:102EE3009E7D9E7D9E7D9E7D9E7D9E9D9E9D9E9DA7
:102EF3009E9D9E9DA69DA69DA69DA69DA69DA69DC7
:102F0300A69DA69DA69DA69DA6BDA69DA69DA6BD66
:102F1300A69DA69DA69DA69DA69DA69DA69DA69D96
:102F2300A69DA69DA69DA69DA69DA69DA6BDA69D66
:102F3300A6BDA6BDA69DA67DA67DA67DA67DA67DD6
:102F4300A67DA69DA67DA69EA6DEA71EA71EAF1ED6
:102F5300BF3EC73EAEDEA69DB6FEBF3ECF3FD73FC8
:102F6300D71EDF3FE77FE77FE79FEFBFEFBFEFBFEF
:102F7300EF9FEFBFEFBFE77FE75FDF3ECF3ED79F18
:102F83006D9B03FA049E049F049F0C9E04BE04FFE2
:102F930004DE04DE04DE04DF0C3C75FCD75FCEDF09
:102FA3005CBB7D9D755C64FB5C9A4C3944394C3940
:102FB3006D1C8E1E755C6D1B549A447A4C7A85DEAB
:102FC300961E7D5C6D1B549A5CDA8E3F8E3F755C5A
:102FD30064DA64FB965F963F7D7C64DA85BD965F19
:102FE3008DFE6D1B85BD963F8DDD95FE8DDD95FEBA
:102FF3008DFE859D8DDE8DFE7D9C7DDE7D9E757DAA
:10300300755D6CFC753C6CFA84947BEF84D664FA32
:103013005D3E4C9B4C9B4CBC4C9C4C9C4CBC4CBC5C
:103023004CBC4CBC4C9C4C9C4C9C4C9C4C9C4C9C1D
:103033004C9C4C9C4C9C4C9C4C9C4C9C4C9C4C9C4D
:103043004C9C4C9C4C9C4C9C4C9C4C9C4C9C4C9C3D
:103053004C9C4C9C4C9C4C9C4C7C4C7C4C7C4C7CAD
:103063004C9C4C9C4C9C4C9C4C9C4C9C4C9C4C9C1D
:103073004C9C4C9C4C9C4C9C4C9C4C9C4C9C4C9C0D
:103083004C9C4C9C4CBC4C9C4CBC4CBC4CBC4CFD1C
:103093004CFD551D551D551D4D1D4CFD4CFC4CFD4A
:1030A3004CFD4CFD4CFC4CDC4CDC54DC54FD54FD21
:1030B30054FC4CFD551D4D1D4D1D553D553D553D78
:1030C300553D553D553D551D551D553D551D54FC0F
:1030D30054FC54DC54DC54DB54DC54DC54DC54DC4E
:1030E30054DC54DC54DC54DC54DC54DC54DC54DC5D
:1030F3005CDC54DC5CDC5CDC54FC54FC54DC54DCF5
:1031030054DC54DC54DB5CDC5CDC5CDC5CFD5D1DB2
:103113005D1D54FC54FC553C553C551B54FB5D1C38
:103123005CFC5D1C5D3D5D1C5D5C65BD6DDD863ECF
:103133009E7EA67EA69FA67FA65EAEBFB69FAE5E10
:10314300B65EC6DFD71FD75FDF7FE77FE77FE77F07
:10315300E79FE79FDF5FD71ED71ECEFFC6DFBE9E6A
:10316300BF1F54FA0BFA04BF04DF04BE049E049F7E
:1031730004BF04DF04FF04DF0C5C65DCAEFFAE5D5F
:103183004C388E1EAEDFAE9FA63D8DDB7D9B6CFB68
:103193006CFBA69FA6BFAE9FA61E85DE755C8DBD8C
:1031A300AE5EAE7EAE7F9E3E85BC7D7B963E9E7FB1
:1031B3009E7F963E7D7C7DBC965E9E7F85DD753BC6
:1031C3007D9C965F859C64DA6D3D85DF64FC64DBE2
:1031D3006D5D5CDB5CDB651C5CFC5CDC5CFB64FAEE
:1031E3008DFBB69CAE7BB69CC65AC659955A755D87
:1031F30075BE655C54BB4CBC4CBC4CBD4CBD4CBD9E
:103203004CBD4CBD4CBD4CBD4CBD4CBD4CBD4CBD73
:103213004CBD4CBD4CBD4CBD4CBD4CBD4CBD4CBD63
:103223004CBD4CBD4CBD4CBD4CBD4CBD4CBD4CBD53
:103233004CBD4CBD4CBD4CBD4CBD4CBD4CBD4CBD43
:103243004CBD4CBD4CBD4CBD54BD54BD4CBD4CBD23
:103253004CBD4CBD4CBD4CBD4CBD4CBD4CBD4CBD23
:103263004CBD4CBD4CBD4CBD4CBD54DD54DD4D1E61
:103273004D1E4CFD4CFE4D1E4D1E4CFD4CFD44FDA4
:10328300451D4D1D4D1D4D1D4CFD4D1E4D1E4D3EF1
:103293004D3E4D3E4D5E4D5F4D7F4D7F4D7F4D7F8E
:1032A3004D7F4D5F4D5F4D3F4D3E4D1E44FE4CFEE9
:1032B3004CFE4CDE4CDE4CDE4CDE44FE4CFE4CDE63
:1032C3004CDE4CDE44DE44DE44DE44DE44DE4CDED3
:1032D3004CFE4CFE4CFE4D1F4D1F44FE44DE44DEAF
:1032E30044DE44DE4CDE4CDE4CFE4CFE4D1F4D1FD7
:1032F3004D3F4D1E453E457F4D7F455E451E4D3F2F
:103303004D3F451F44FE44FE451E559F6DFF7E1EE7
:10331300963EA67FA69F963E8DFD961E963E963FB1
:103323009E5FA67FB6BFBEDFBEDFC6DECEFED71E64
:10333300DF1FD71FD71FCEFFCEFFC6DFC6FFBEBF1F
:10334300BE9EBEFF44B9041A04DE04DF04BF0C9F13
:10335300047F049E049E049F0C3C55BD96BF9E3E75
:1033630095BC95BC9DFDA63EAE9FB6BFB6BFAE9EB7
:10337300961D751B7D9D8DFE9E5EAE7EAE9F85DE8A
:103383005CBB653D7DDE961E9E7F6D5D54795CDB87
:103393006D3C861F757D4C7A549A5CDB757D64FBAE
:1033A300549A549B5CDC64FC5CBB5CBB757D759E72
:1033B3005CDB653D7DFF755E757E861E85DE7D7BF0
:1033C300BEDCFFFFFFFFFFFFFFFFFFFF8D7B755D90
:1033D3006D5D6D7C5CFB4CBC4CBC4CBC4CBD4CBDB6
:1033E3004CBD4CBD4CBD4CBD4CBD4CBD4CBD4CBD92
:1033F3004CBD4CBD4CBD4CBD4CBD4CBD4CBD4CBD82
:103403004CBD4CBD4CBD4CBD4CBD4CBD4CBD4CBD71
:103413004CBD4CBD4CBD4CBD4CBD4CBD4CBD4CBD61
:103423004CBD4CBD4CBD4CBD4CBD4CBD4CBD4CBD51
:103433004CBD4CBD4CBD4CBD4CBD4CBD4CBD4CBE40
:103443004CBE4CBE4CBE4CDE4CDE54DE54FF4CFE38
:103453004CFE4CFE4CFE4CFE4CFE4CFE4CFE4CFE19
:103463004CFE4CFE4CDE4CDE4CFE4CFE4D3E4D5EA7
:103473004D5E4D5E4D7F4D9F4D9F4D7F4D7F4D5E0C
:103483004D5F4D5E4D3E4D3E4D1E4CFD4CFD4CFD86
:103493004CFD4CDD4CDD4CFD4CFE4CFE4CFE4CFE1D
:1034A3004CFE4CFE4CFE4CFE4CFD4CFD4CFE4CFECB
:1034B3004CFE4CFE4D1E4D1E4D1E4D1E4D1E4D1EF3
:1034C3004D1E4CFE4CFE4CFD4CFD4CFD4D1E4D1E49
:1034D3004D1D4D3E553E655D659D75DE6DDE657E1C
:1034E3004D1C555D5D7E5D5D5D7D659D75FE967FC5
:1034F300A69FA69E9E7F8E1D85BC85DD8E1E8E3F5C
:10350300861F85FE8E1E963E9E3EA63EAE7EB67EF0
:10351300BEBFC6BFC6BFC6DFC6FFC6FFBEDFB69E01
:10352300AE5DAE9E9E7E3C392CBD14BE04BD04BC74
:1035330024FC2CFC24DC34DD2C7B657C8E5F8DDE4F
:10354300B6DF751A54385CBA6D1C7D7D8DBD9E5EE9
:103553009E7F6CFB4C3A4C7B4C9A751B7D9D75BED4
:1035630054DC4C9B4C7A549A5CDB6D5E6D5D5CDB8A
:10357300547A4C5964FC7DDF759D6D1C547A7D9D96
:10358300965F7D9D6D3C85BE9E5F95FD8DBD95FED1
:10359300963F963F859C7DBC863E6D9C6D9C755B7E
:1035A300B67BFFDFFF9EFFBEF7BFE7BF7D186D1B36
:1035B300653C755D6D7D54FC4CBC4CBC4CBD4CBD39
:1035C3004CBD4CBD4CBD4CBD4CBD4CBD4CBD4CBDB0
:1035D3004CBD4CBD4CBD4CBD4CBD4CBD4CDD4CDD60
:1035E3004CDD4CDD4CDD4CDD4CDD4CDD4CDD4CDD90
:1035F3004CDD4CBD4CBD4CBD4CBD4CDD4CBD4CBD40
:103603004CBD4CDD4CDD4CDD4CBD4CBD4CDD4CDDCF
:103613004CBD4CBD4CBD4CBD4CBD4CBD4CBD4CDD3F
:103623004CDD4CDE4CDE4CDE54FE54FE4CDE4CFED8
:103633004CFE4CFE4CFE4CDE4CFE4CFE4CDD4CDD99
:103643004CDD4CFE4CFE4D1E4D1E4D3E555E555EF3
:103653004D7E4D7E4D7E4D9F4D9E4D7E4D7E4D5DEF
:103663004D3D4D3D4D1D4D1D4D1D4D1D4D1D4D1DC7
:103673004D1D4CFD54FD54FD4CFE4CFE4CFE4CFECA
:103683004CFE4CFE4CFE4CFD4CFD4CFE4CFD551EC1
:103693004D1E4CFD4CFE4D1E555D557E557E557E93
:1036A300557E557E4D3D4D1D4CFE4CFE4D1E4D1E13
:1036B3004D1E555F5D9F7DFF8E7F96BF8E7F75BDCF
:1036C3006D7B7E3E969F8E3E967F967F969F9EBF96
:1036D3009EBF9E7EA6DFA6DF965E965E967F9E9F2A
:1036E3009E7F7DDD6DBD75DE861F8E3F965F9E5F7F
:1036F300A67F9E9F9E7F9E7FA67FA67FA63EA61D3A
:103703009E3D9E3EA65E961E5D5D4DDF147B2D5D48
:103713007EBF8EBF865E865F7DDE7DDD861D85DE98
:10372300965F757D54BA4C9A447A447A4C9B5CDD1F
:103733006D1D85BD757C64FB54DD449C447A64DA5D
:103743009E3E9E3E85BD755D5CBA64DAA69FA69FCC
:103753009E5E8DFD7D5B961EA69FAEBF9E5E95FD14
:103763008DBC9E5EA69F9E5E6D3B7D9D967F7DBDBF
:1037730064FB6D3B757D64DA5CDB655D6D7D64D9EF
:10378300B69CFFFFFFFEFFDEFFFFF7FFA65C8E3E4A
:1037930085DE759E75BE5D5D4CDB54DC54FD54DDEA
:1037A30054DE54DE4CDE4CDE4CDE4CDE4CDE4CDEB6
:1037B3004CDE4CDE4CDE4CDE4CDE4CDE4CDE4CDEB6
:1037C3004CDE4CDE4CDE4CDE4CDE4CDE4CDE4CDEA6
:1037D3004CDD4CDD4CDD4CDD4CDD4CDD4CDD4CDD9E
:1037E3004CDE4CDE4CDE4CDE4CDE4CDE4CDE4CDE86
:1037F3004CDE4CDE4CDE4CDE4CDE4CDE4CDE4CDD77
:103803004CDD4CDD4CDD4CFE4CFD4CFE4CFE4CFDCA
:103813004CDD4CDD4CDD4CDD4CDD4CDD4CFE4D1EFA
:103823004D1E4D3E4D3E4D5F4D7F4D7F4D9F4D7F18
:103833004D9F4D9F4DBF4DBF4DBF4DBF4D7F4D5E06
:103843004D5E4D5E4D3E4D5E4D7F559F557F4D5FA9
:103853004D5F4D3F4D1F4D1F4D1E4D1E4D1E4D3E89
:103863004D3E555E5D9E5D9E657E657E6DBE657D4E
:103873005D5D5D5D553D4D5D4DBF4DBF55BF559E76
:1038830055BF55DF4D7E4D3E4D1E4D1E4D1E4D1EEB
:103893004D3E555F4D5E4DBE55BE5DDE761F7E1EB1
:1038A3007E1F8E9F9E9F9E7F967F863F7E1E761EE7
:1038B300761E7E5F8E9F967F967F967E9E9F9E9FAF
:1038C3009E9F8E5E761E6DFE6DDE75DE7DFF7DFF37
:1038D3007DFF75FF6DDE75DE7E1F861E963F9E5F44
:1038E3009E5F9E5FA67E965D6DDC247934FC5DDF72
:1038F3007DBE8DFE8DFE95FF8DFF8E3E861F7DFF67
:103903006CDB9E1EAEDE9E5D8E1E85FE757E6CFD9F
:103913006CDB95FDBF1FB6BEB6BF965E8DFE85BC44
:10392300A65EBEFFBF1FBEFFB6DFA69E95FC9E1C14
:10393300A69EB6DFBEFF9DFD7D5B8DFD963E9E9FE1
:103943007D9D6D1B757D861E7DFE759D653C7DBDD4
:103953008E3E85DD7D9C9E5E9E5F961EA67EAE7E20
:10396300BF1EBEFDC6DCCF1EC6BC5AEB29A9320E54
:103973007D3B759D6D5C75DE655D5D3D553D553EDD
:103983005D1E5D1D551E551E551E551E54FD54FDD1
:1039930054FD54FE54FE54FE54FE54DE4CDD4CDE06
:1039A3004CDE4CDD4CDD4CDD4CDD4CDD4CDE4CFEA9
:1039B3004CFE4D1E4CFE4CFE4CDD4CDD4CDD4CDD17
:1039C3004CDD4CDD4CDD4CDD4CDD4CDD4CDD4CDDAC
:1039D3004CDD4CDD4CDD4CDD4CDE4CDE4CDD4CFE79
:1039E3004CFE4CFE4CFE4CFE4CFE4CFE4CFE4CFE84
:1039F3004CFE4CFE4CFE4CFE4CFE4CFE4CFE4D1E53
:103A03004D3E4D3F455F4D7F4D5E557E559F55BFA6
:103A13005DDF65FF5DDE55BE4DBE4DBE55BE559E99
:103A23004D9F4D7F4D5F455E4D7E4D7E4D3E4D1D01
:103A33004D1E4D1E4D3F4D3F453F4D3E4D3F4D3F6E
:103A43004D3F4D5E5D7D861EB6BFBF1FC71FBEFFC8
:103A5300BF3FAF1F865D6DDD5DDE7E3F863F75FE3A
:103A63005DBD55DE55BF4D5E4D5F4D3E4D3E4D3EFA
:103A73004D1E4D3E4D3E4D5E4D5E557E65FE6E3F89
:103A83006E3F661E65DE6DFF65FF5DDE55BE4DBD97
:103A93004D9D55FE65FF6DFE7E1E8E3E967E967F86
:103AA3008E5F865F7E5F761E6DFE65FE5DFF5DDF6A
:103AB30055DF55BF559F65DF761F7E1F8E5F967F4F
:103AC3008E5F863F861E75FD6E1F3CFC349A4D5DEE
:103AD3007E1F965F9E3FAE7FAEBF7DFD5D7D557EB3
:103AE3005438859CB6FFBEFFBEBFBE9FAE7EA61DEB
:103AF30095DD95BC9E3EA67EAE9FBEBFBEBEBEDF1D
:103B0300859B6CFA7D7D85FE9E7FAE7F7D7D4C5AC5
:103B13004C9C5D1D6D5D6D5E54DE4C9C4C7A54BABD
:103B23006D9D7DDE64FD5C9B7D3B9E5F8DFE85BD53
:103B3300963F9E7F9E5F85FD757C8E3E7DBD64FBBB
:103B43006D7D5D1D54BC5CDD7CB94A07000000003F
:103B53008D58863D85FE85FF6D9E54DD4CDD4CDE24
:103B63004CDE4CDD4CDD4CDD4CDD4CDD4CDD4CDD09
:103B73004CDD4CDD4CDD4CDE4CDD4CDD4CDE4CDEF7
:103B83004CDE4CDE4CDE4CDE4CDE4CDE4CFE4CFEA2
:103B93004CFE4CFE4CFD44DD4CDD4CDD4CDD4CDD80
:103BA3004CDD4CDD4CDD4CDD4CDE4CDE4CDE4CDEC6
:103BB3004CFE4CFE4CFE4CFE4CFE4CFE4CFE4CFEB2
:103BC3004CFE4CFE4CFE4CFE4CFE4CFE4CFE4CFEA2
:103BD3004CFE4CFE4CFE4CFE4CFE4D1E4D1E4D1E2F
:103BE3004D5F4D7F4D7F4D9F559F5DBF6DFF7E3F69
:103BF300865F863F7E1E7E1E7E1F75FE763F65FFB7
:103C0300559F4D7E4D3D5D3C655C657C657B6DBD23
:103C1300659C5D7C5D9E559E4D7E4D5F451E451E9C
:103C2300453E4D3D65BE969FBF1FCF5FD75FDF5FAC
:103C3300DF5FCF1FC6FFBEFFB6DFB6BFAEBF96BF07
:103C4300767F55DE4D7D559D559C4D5C5DDD65FE56
:103C530065DD6DFD761E6DDE659D659D65FE65FE0C
:103C63005DBE55BE4D9E4D9F4DBF4DBF4DBF4DBE1D
:103C730055DE55DE65DE75FE865E967F969F8E7FEA
:103C8300863F7E3F6E1F65FF65FF5DDF55DF55DFB6
:103C93004DBF4DBF4DBE4DBF55BE559E5DBE5DBEB6
:103CA3005D9E559D557D557D4D7E555E447A85DDE2
:103CB3009E5EAE7EB67EB69EAEBF759D4D1D4D3EDD
:103CC3009E7E85FD8E1D9E3DAE5EBE9FBEDFBEFF0A
:103CD300BF1F9E5E5C9A5CDC651D857D95FD965FCE
:103CE30085DE549B4C5A4C9B54BB64DC6D3E759EE5
:103CF300651D54BB4C7B4CBB963EA67F8DDE74FB8F
:103D0300855CA67FAEBFA69F961E8DBD8E1E9E7F31
:103D13008E5F5CDA6D5C75DE5CFC54BC5CDC6D5DF7
:103D2300653D651C861E7DFE8D5983EC422829AABC
:103D3300859C6D9F6D3D651C653D54FD4CDD4CFEC2
:103D430054FE54FE4CDE4CDE4CDE4CDE4CDE4CDED0
:103D53004CDE4CFE4CDE4CDD4CDE4CDE4CDE4CDEF1
:103D63004CDE4CFE4CFE4CFE4CFE4CFE4CFE4CFE20
:103D73004CFE4D1E4D1E4D1E4CFE4CFE4CFE4CFE8D
:103D83004CFE4CFE4CFE4CFE4CFE4CFE4CFE4CFEE0
:103D93004CFE4CFE4CFE4CFE4CFE4CFE4CFE4D1EAF
:103DA3004D1F4D1F4D1F4D1F4D1F4D1F4D1E4D1EB2
:103DB3004D1E4D1E4D1E4D1E4D1E4D1E4D3E4D5F47
:103DC3004D7F4D9F4D9F4D9F55BE661F863F8E5F16
:103DD3008E5F965F9E7F9E7F965F863F761E65BE53
:103DE300559E65FE865F9E7EB6BEBF1FC73FBF3F23
:103DF300B73FA6FF8E9F6DDD5D7D5D5D655D6D9D4E
:103E03006DBD6DBD85FD9E5FBEDECF1FCF1FCF1F76
:103E1300CF1FC6FFBEDFBEFFB6FFA67F8E1F6DDEC0
:103E23005DDE4D7C65FE96DF9EBE7D9B8DFCA69F71
:103E3300AEDFB6FFAEDF96BF865E7E5F7E7F661F18
:103E430055BF55BF4DBF4DDF4DDF55DF55DF5DDE40
:103E53006E1F763F7E3F863F865F8E5F8E7F7E3FFF
:103E630075FF65FF5DFF55BF55BF4DBF4DBF4D9FEF
:103E73004D9F4D9F4D9E4D9F4D9E4D7E4D7F4D7E43
:103E8300457E457E457E455F455F4D5F64FC95DC21
:103E9300CF3FCEFFCEDDC6BDBEDF7DBC4D1D4D3F4A
:103EA300BF3F967E549A549B5CBC6D3D7D7D7DDC0B
:103EB3008E5E8E7F54FB4C9C4C7C449B4CBC4CBC18
:103EC3005D3D7E1E7DBD7D5C5CFD44BC5CBAA69EF3
:103ED300BEBFAE7E961D85DC95DCAE7EAEDFAEDF6B
:103EE300A6DF757B6D7C7DDE8E7F759D549954DADC
:103EF3006D7D75DE653C54BB759D965F859D8DDD3F
:103F0300A67FA65E95DD8DBC95997C508578757DE1
:103F13005D3D54FD755C7DBD7DFF75FE551D4CFDFE
:103F23004CFE4CFE4CFE4CFE4CFE4CFE4CFF4CFE3D
:103F33004CDE4CFE4CFE4CFE4CFE4CFE4CFE4CFE4E
:103F43004CFE4CFD4CFE4D1E4D1E4D3E4D3E4D3E1A
:103F53004D5F4D5F4D3E4D1E4D1E4CFE4CFE4CFEC7
:103F63004CFE4CFE4CFE4CFE4CFE4CFE4D1E4D1EBC
:103F73004D1E4D1E4D1E4D1E4D1E4D1E4D1E4D1EE6
:103F83004D1F4D1F4D1F4D1F4D1F4D1F4D1E4D1ED0
:103F93004D1E4D1E4D1E4D1E4D3E4D3E4D5F4D7FE4
:103FA3004D7F4D7F4D7F4D7E557D5DBD7DFD8E5E8D
:103FB300965E9E9F9EBF8E5E861E861E861E7E1EFC
:103FC300863E969FA69FC71FD73FD6FED6FECEFE40
:103FD300CF1EC71FB6DF9E3E965E9E7FAE9FB6DFA7
:103FE300AEDFA6BFA69FAE5FAE7FAEBFA67F965FD6
:103FF3008E5F7E5F763E6E1E65BE5D7E553E4D5F77
:104003004D7E559E761E969F9EBF969F969F967F4A
:104013009E9F9E9F8E5E7E3E6DDD65DD661F5DFF0E
:1040230055BF4DBF55DF5DDE5DFE661F6E3F7E5F94
:10403300867F865F7E3F761F6DFE6DDE6DFF661F9A
:104043005DDF55BF4DBF4DBF4DBF4DBF4D9F4D9F15
:104053004D7F4D7F555F557F4D7F4D5F4D5F4D5F6D
:104063004D3F4D3F4D3F4D3F453F453F553C64F927
:10407300A63CDF7FE79FDF5FC73F85DC4CFD4D3FFD
:10408300A69E965E64DC549C449C449B449C4C9C3E
:1040930054BC651C9E7F963E85BD6D5C653C5CFB98
:1040A3005CB99E9EBF3FBEDFAE9F9E7E963E8DDD7A
:1040B3009E5EA67EAEDFB71F8E3F5CDB651C6D7D0B
:1040C300865E6DBD4CDC4C9C54DB5D3C863F759C31
:1040D30064FA8DFDA6DF9E7F963E8DFD965E967FEC
:1040E3006D3C64DD6D3D6CFC747773EF8D996D5C95
:1040F30075FE865E963E861E7DDE657D5D5E4CDDCD
:104103004CFE4CFE4CFE4CFE4CFE4CFE4D1E4CFE3B
:104113004CFE4CFE4D1E4D3E4D1E4D1E4D1E4D1E66
:104123004D1E553E553E4D3F4D5F555F555F4D5FAF
:104133004D5F4D3E4D3E4D1E4D1E4D1E4D1E4CFEC4
:104143004D1E4D1E4D1E4D1E4CFE4D1E4D1E4D1E35
:104153004D1E4D1E4D1E4D1E4D1E4D1E4D1E4D3FE3
:104163004D3F4D3F4D3F4D1F4D1F4D1F4D3F4D3E4D
:104173004D3E4D3E4D3E4D3E4D3E4D3E4D3E4D5EC4
:104183004D5F455F4D7E557E5DBE763F8E5F9E7F64
:104193009E9F9E9F967F861E7E1E867F8E5F9E9F1E
:1041A300B6FFC6FFCF1FCF3FD75FCF3FCF1FCF1F76
:1041B300D71FCF1FC6FFBEFFB71FAEFFAEBFA67E82
:1041C300967E8E9F8E9F8E5F7E5F6DDE65DE5DBF0A
:1041D300557E559F4D5E455E453E4D1F4D1F4D5FC0
:1041E300457E4D9E557E5D9E55BE5DBE55BE4D9D25
:1041F30055DE5DFE55DE55DF55FF55FF55DE55FF98
:1042030055DF55DF5DFF661F663F663F661F661F0E
:1042130065FF65FF5DFF5DFF5DFF55DF4DDF4DDF33
:104223004DDF4DDF4DBF4DBF4D9F4D9F4D9F4D7F8B
:104233004D7F4D5F4D5F4D5F4D5F4D5F4D5F4D3E1C
:104243004D3F4D3F553E553E4D3F453F4D3E551C21
:1042530074F8C6FEDF9FDF7FD79F85BC4CDD4D1F03
:10426300549A6CFB9E5F961E85BC75BC655C5CDCDA
:10427300547C649AA67EC71FC6DEBEDFB6DFA69E49
:10428300963C8DDD95DD9E3EB6BEBEBEB6FF85FE79
:104293004C9B54DC5D1D75BE75FE655D54BC549C22
:1042A300547B5CFB965F861E759D6D5C8E3EA6DF20
:1042B300A6BF9E7E859C7D9E8E3F6D7C549B5CDB62
:1042C30085FC963D961CB6DEC6BCB5D69DDA8E1E21
:1042D300863F6D7D757D653C5CFB655D659E54FD2C
:1042E3004CBE4CDE4CDD4CDD4CDD4CDD44DD4CFD89
:1042F3004D1E4D3E4D3E555F553F4D3E4D1E4D1F90
:104303004D1F44FE451E4D1E4D1E4D1E4D1E4D1E82
:10431300451E44FD451E451E451E44FF4CFF4CFFF4
:104323004D1F4D1E4D1E4D1E4D1E4D1E4D1E4D1E31
:104333004D1E4D1E4D1E4D1E4D1E4D1E4D1E4D1F21
:104343004D1F4D1F4D1F4D1F4D1F4D1F4D1F4D3FEA
:104353004D3F4D3F4D3F4D3F4D1E4D1E451F453F6C
:10436300453F453E4D7F55BF5DBF6E1F7E3F863F38
:104373007E3F761E6DDD65DD6E3F765F761E7DBD0D
:104383009E7EB6DFBEDFC6FFC71FBF1FBF3FB6FFA0
:10439300AEDFAEFF9E9F967F865E7E5E761E6DBD10
:1043A30065DD5DDE55BE559E4D9E4D9E4D7E4D7F1A
:1043B3004D5F4D3F4D5F4D3F4D3E553E553E4D5F2D
:1043C3004D7F4D9F4D7F4D7F4D7F4D7F4D9F4D9F2A
:1043D3004DBF4DDF4DBF4DDF4DDF4DDF4DDF4DDFBA
:1043E30055DF55DF55BF55DF55DF4DBF4DDF4DDF82
:1043F3004DBF4DBF4DBF4DBF4DBF4DDF4DDF4DDFFA
:104403004DDF4DBF4DBF459F4D7F4D7F4D7F4D7F51
:104413004D7F4D5F4D5F4D5F4D5E4D5E4D5E455E25
:10442300453F4D3F555E551D4D1E451E451E551DB1
:104433005CB88D79D73FC71EAEBD85DC5CFB4CFDF8
:104443005CBC64DBB6FFCF5FCF1ECF3EBF1FB6BEE3
:10445300A65E9E3E9E1DAE9FB6DFBEFFBF1FC71F5B
:10446300C75F961D5CDA653C6D7D7D9D85DE8E3F65
:10447300755D64FD64FD5CFD5CFB8E3EA6DF9E5DA9
:104483009E3E857BA67EB73FBF1FBF3FA65D857B54
:104493008DDC9E9E965D64DA651B75BC967E8DDC15
:1044A300C6DDFFFFFFFFFFFFFFFFFFFFAE9D755A56
:1044B300757B85FD7D7C859D9E5F9E5EA69F965F39
:1044C300757C655D657D5D7D5D7D5D7D5D7D5D9DF2
:1044D30065BE65DE65FE65FE65DE65BE659E659E41
:1044E300659E5DBE659E659E659E659E659E659E99
:1044F300659D659D659D657D659E5D9E5D9E65BEB5
:1045030065DE65DE65DE65BE659D659E659E5D9EB9
:104513005D7E5D7E5D7E5D9E5D9E5D9E5D9E5D9E20
:104523005D9E5D9E5D9E5D9E5D9E5D9E5D9E5D7ED0
:104533005D7E5D9E5D9E5D9E5D9E5D9E5D9E559EC8
:104543005DBE5DBE65FF663F5DDE5DDD5DBD5DDE5F
:104553005DDE5DDE5DDE65FE65DE65FE65DF5D9D60
:10456300659D863E9E9FA6BFA69E9EBF967E863E67
:104573007E3E761E65FE5DBD55BE55BE55BE559E3F
:1045830055BE55BE55BE55BF559F559F559F4D7E34
:104593004D5E4D7E4D5E4D7E55BF559F4D9F4D9F4C
:1045A3004D9F4D9F559F4D9F4D9F4D9F4D9F4D9FA0
:1045B3004D9F4D9F4D9F4D9F4D9F4D9F4D9F4D9F98
:1045C3004D9F4D9F4D9F4D9F4D9F4D9F4D9F4D9F88
:1045D3004DBF4D9F4D9F4D7F4D7F4D7F4D9F4D9FB8
:1045E3004D9F4D9F4D9F4D7F4D7F4D7F4D7F4D7E09
:1045F3004D5E4D5E4D5E4D5E4D5E4D5E4D5F4D3F7E
:10460300453F4D5F4CFC5D1C6D7C75FE7E1E8E3EF2
:10461300861D7D39ADFCB73F759B965CC75FA67E53
:1046230095FD95DDAE7DBEFECF3ECF3ED73ED73E58
:10463300D73FCF5F9E5E653B6D9E6DBD75BC8E1D86
:104643009E5E9E3E7DDD6D9D5D7C5D7B655B757BCA
:10465300AEDEB71EBEFDB69D963C9E3CBEDDCF3E94
:10466300CF3ECF5FAEBD859A85DC965D9E7D85DCB2
:104673007D7B757A8DFBB71EAEFD9E7CA67DB6DE77
:10468300DF7EF7BFF79EF7DFF7DFE79E9DF9963BE7
:10469300A6BDA67CAE9DB6DEA65C95FB95FB85FB11
:1046A3007D9C75BC75DC75DC75DC75DC7DDC7DFCA7
:1046B3007DFC7E1C761C7E1C761C75FC75FC7DFCCB
:1046C3007DFC85FC85FC7DFC7DFC7DFC7DFC7DFC0F
:1046D3007DFC7DFC85FC85FC85FB861B863B863B40
:1046E3007E1B7E1B75FB75FC75FC75FC75FC75FCF0
:1046F3006DFC6DFC6DFC6DFC6DFC6DFC6DFC6DDC8F
:104703006DDC6DDC6DDC6DDC6DDC6DDC6DDC6DDD5D
:104713006DDD6DDD6DDD65DD65DD6DDD65DD65FD46
:104723006E1D6E1D6E1D65FC65FC6E3D6DFE65BEEA
:1047330065BE65BE65DE65BE659E5DBE5DDE5DDE36
:104743005DBE65DD761E763E761E6E1E65FE65DEFB
:104753005DDE5DDE5DFE55FE55FE55DE55DE55DE46
:1047630055DF55DF55DF55BE55BF55BE559E559E8A
:104773004D7E4D7E4D7E559E55DF55BF4D7F4D9FE2
:104783004D9F4D9F4D9F4D9F4D9F4D9F4D9F4D7FE6
:104793004D7F4D7F4D5F4D5F4D5F4D5F4D5F4D5F76
:1047A3004D5F4D5F4D5F4D5F4D5F4D5F4D5F4D5FA6
:1047B3004D5F4D5F4D5F4D5F4D7F4D7F4D5F4D5F56
:1047C300455F4D5E555E555E4D5E555F4D5F4D5E7B
:1047D3004D5E455F455F4D5F4D5F4D3F4D3E4D3EE9
:1047E3004D3E4D3D861DBF1ED77FCF3FCF1FBEBE63
:1047F300C6DFC6DE74F85D7D2C998E5BEFFFDF1E8E
:10480300C71FBF1F751A6CFB757E759D85BD961DF1
:10481300A67DB6FF965D54BA4CBB44BC44DD4CBD8B
:104823004C9D651DA69FAE9E9E5C8E5D85BD74FBF3
:104833008DDDB6FFB71FB73FBF1FB6DE6D3A6D7C88
:104843006DBE75FE8E5E655C44DD4CDC4CBA75FD59
:10485300969F85FD8DDDA67FA69EAEFF963E6CB727
:10486300B6BBFFFFF7DFFFDFFFDFFFFFB69C9E5EF8
:10487300963F9E7F7DDE5D3E5D3C653C653C7DFEF7
:104883007E1F5D1D4CDD4CDD4CDD4CDD4CFD4CFDD8
:104893004CFE4D1E4D3E4D3E4D3D4D3D4D3E4D5E00
:1048A3004D5E553D4D3D4D3E4D3E453E4D3E4D5E6F
:1048B3004D5E453E4D3D5D7D75DE863F863F7E1EEA
:1048C30075FE65BE5D9E4D5E453E453E451E4D1ED5
:1048D3004D1E4D1E4D1E4D1E4D1E4D1E4D1E4D3E5D
:1048E3004D3E4D3E4D3E4D3E4D3E4D3E4D3E4D5E4D
:1048F3004D5E4D5E4D5E4D5E4D5E4D5E4D5E4D5E5D
:104903004D5E4D5E4D5E4D5D4D5D4D5E4D5F4D3E6D
:104913004D3E555F4D3E4D3E555F4D5E4D7E4D9E2A
:104923004D9E55DE55FF55FF55DE4DBE4DBF4DBF68
:104933004DBF4DDF4DDF45BE4DBE4DBE4DBE4DBFE0
:104943004DBF4D9F4D9F4D9F4D7F4D7F4D5F4D5EA5
:104953004D5E4D5E4D5F4D7F4D7F4D7F4D7F4D7F56
:104963004D7F4D7F4D7F4D5F4D5F4D5F4D5F4D5F84
:104973004D5F4D5F4D5F4D3F4D3F4D3F4D3F4D3F74
:104983004D3F4D5F4D5F4D5F4D5F4D5F4D5F4D5FE4
:104993004D5F4D3F4D5F4D5F4D5F4D5F4D5F4D5FD4
:1049A3004D5F4D5F4D5F4D5F4D5F4D5F4D5F455FAC
:1049B3004D5F4D5F4D5F4D3F4D3F4D3F553E4D3E2E
:1049C300553D7DFDCF9FEF9EE73DD6DDC69DBE7D68
:1049D300CE9EDF5F7D9A03D80CBC6E7CD79FDEDE54
:1049E300CF5FBF5F757C4CBC4CDF44DF44DD4CFDC7
:1049F300551D5D1B759C9EBF963D85DD759D657E32
:104A03005D3D5CFBA6BECF5ECF5EC75FBF3FB6FF1B
:104A1300963E6D3A6DBC7E3E9E7E9EBF6DDE44FD2E
:104A23003CFE44DD4CFC865E9EDF967F85BD7D7C2F
:104A3300A69EB6DEBF1FA69F64FB653D75BE757B54
:104A4300A6BCCF7ECF1DDF9FF7BE7BCF52EC539228
:104A5300759C5D3C5D5C6DBE6D7C863E9EBF967EA7
:104A630085DD7DDD4D3E4D3F4D3F4D3F4D3F4D3F40
:104A73004D3F4D3F4D5F4D7F4D7F4D9F4DBF4DBFD3
:104A83004D9F4D9F457F459F45BF4DBF4DBF5DDF4B
:104A930065DE7E1E967FA6BFAEBFB6BFAE7FA67F86
:104AA300A69F969F865F6DDF5D7E555E555D555E65
:104AB3004D7F4D7F4D7F4D7F4D7E4D7F4D7F4D7F94
:104AC3004D7F4D7F4D7F4D7F4D7F4D7F4D7F457F8B
:104AD3004D9F4D9F4D9F4D9F4D9F4D9F4D7F457FBB
:104AE300457F457F457F457F457F457F4D7F4D7F93
:104AF3004D7F4D7F4D7F4D7F4D7F4D7F4D9F4D9F13
:104B03004DBF4DDF4DFF4DDF4DDF4DDF4DDF4DBF62
:104B13004DBF4DDF4DDF4DDF4DDF4DDF4DDF55DF4A
:104B23004DBF4DBF4D9F4D9F4D7F4D5F4D5F4D7FA2
:104B33004D5F4D5F4D5F4D7F4D7F4D7F4D7F4D7F72
:104B43004D7F4D7F4D7F4D5F4D5F4D5F4D5F4D5FA2
:104B53004D5F4D5F4D5F4D5F4D5F4D5F4D5F4D5FF2
:104B63004D5F4D5F4D5F4D5F4D5F4D5F4D5F4D5FE2
:104B73004D5F4D3F4D5F4D5F4D5F4D5F4D5E4D5EF4
:104B83004D5F4D5F4D7F455F455F4D3E4D7F557E8C
:104B93004D3E4D3D555E555F4D3F4D3F555F4D3E3F
:104BA3006DDEA6DFCF5FDF3ED6FDCEFECF1FCF1F6C
:104BB300D73FDF1EBF1F34B90418661CAF1FBE9F4B
:104BC300861C8E3D85FE655D5D1D54FC4CFD4CFED3
:104BD30044DF44BD653CB71FC75FCF3FC71FBF1F3F
:104BE300B6FF9E9E8E3D861E8E1EA67EB6FFB73FE7
:104BF300A6FF5CFB4CBC4CDE4CFE4CDC75DE9E9F82
:104C03008DFE8DFE7D9D85BCBEDFBEFFBF1FB71F22
:104C1300757C651B6DBE7E3E7E1E655D54FD75BD58
:104C2300AF1FAE9E9E3D8DFCA5B941C8000000029A
:104C33006CB87E1E7DFD965E9EBF9EBF7D9C759D5E
:104C4300657D5D7E4D1E4D3F4D3F4D3F4D3F4D3F7D
:104C53004D3F4D5F4D5F4D7F4D9F4D9F4DBF4DBFB1
:104C63004DBF4D9E4D9E4D9E4D9E5DBE6E1E865FFD
:104C7300967EB6DFBEFFC6FEBEDEB6BEA6BF969F5D
:104C8300865E6DFD5DBE4DBF45BF45BF4DDF55BE65
:104C9300559F4D9F4D7F4D7F4D7E4D7F4D5F4D7F8A
:104CA3004D7F4D7F4D7F4D7F4D7F4D7F4D7F4D7FA1
:104CB3004D7F4D7F4D7F4D7F4D7F4D7F4D7F4D5FB1
:104CC3004D5F4D5F4D7F4D7F4D7F4D7F4D5F4D5F01
:104CD3004D5F4D7F557F4D7F4D7F4D7F4D9F4D9F49
:104CE3004D9F4DBF4DDF4DBF4DBF4DDF4DBF4DBF41
:104CF3004DBF4DBF4DBF4DBF4DDF4DDF4DDF4DBFF1
:104D03004DBF4D9F4D9F4D7F4D7F4D7F4D7F4D7FC0
:104D13004D7F4D7E4D7E4D7F4D7F4D7F4D7F4D7F32
:104D23004D7F4D7F4D7F4D5F4D5F4D5F4D5F4D5FC0
:104D33004D5F4D5F4D5F4D5F4D5F4D5F4D5F4D5F10
:104D43004D5F4D5F4D5F4D5F4D5F4D5F4D5F4D5F00
:104D53004D5F4D5F4D7F4D5E4D5E557E557E5DDFF4
:104D6300557D4D5D559E5D9E5D9E6DDE6DBD7DFEEB
:104D7300865E763E659D553D555F4D5F4D5E4D9E0E
:104D830065BE8E3FA69FB6DFB6DFB6FFBEDFC6DECB
:104D9300BEBEBE7DC6BE7D9A3C158E3DB6BFB67EF9
:104DA3004CDE54DD965FBF3FBEFEB6DEA6DE9E7EC2
:104DB3008E1E7D9D757CA67EB6FEBF1FCF3FD73F5F
:104DC300CF5ECF7F965E54DD4CDF54FE5D5E659D06
:104DD3006D9C861E7DDE757D657D5D5D6D3CA6DF0C
:104DE300C77FC75FC71FB6DF7D9C6D5D75BE7E5EE7
:104DF3007E7F5D7C5D3D54FB7E1CAF3FA6BF9E9FC7
:104E03008E3D8E3D9EFF75FD7475838C28E421696C
:104E130085DB8E7D9EDE96BF75DD655B657D6D9E54
:104E23006DBD8EBF867F5D5C553D4D5F4D3F4D3FF4
:104E33004D3E4D5F4D5F4D7F459F459E4DBE55BEDB
:104E43005DBE5DDE5DBE559E65BE7E1E9E7FB6BFAA
:104E5300C71FCF1FCF1ECF1EC71FBEFFAEFF9E9F14
:104E63008E5F7E3F65DE55BE55BF4DDF4DBE4DBEE9
:104E73004D9F4D9F4D7F4D7F4D7F4D7F4D5F4D7EB0
:104E83004D7E557E557F4D7F4D7F4D7F4D9F4D7F91
:104E93004D9F4D7F4D7F4D7F557F4D7F4D7F557F7F
:104EA300557F4D7F4D7F4D7F4D7F4D7F4D9E4D9E59
:104EB3004D9F4D7F4D7F559F559F559F4D9E4D9FB8
:104EC3004D9F4DBF4DDF45BF4DBF4DDF4DBF4DBE68
:104ED3004D9E4DBF4DBF4DBF55BF55BF55BF55BF70
:104EE3004DBF4D9F559F557F4D7F4D7F4D7F4D7FCF
:104EF3004D7F4D7F4D7F4D7F4D7F4D7F4D7F4D9F2F
:104F03004D9F4D9F4D9F4D7F4D7F4D7F4D7F4D7FDE
:104F13004D7F4D7F4D7F4D7F4D7F4D7F4D7F4D7F2E
:104F23004D5F4D5F4D7F4D7F4D7F4D7F4D5F4D7F7E
:104F33004D7F4D7F4D7F4D7F4D9F4D5E6E1F9EFF7D
:104F43009E7E8E1D7DFD8E5F8E3E967F8E1D9E9F67
:104F5300AEFFA6DF863E659D4D7E4D7F4D5F559F1F
:104F63005DBE6DBE6DDE7DFF7DFF8E1F9E1EAE3E60
:104F7300B67EBE9ECEDED73F9579AE5CC71FA67EBA
:104F830054DC5CBA9DFCD75FD75FDF5FDF5ED77F02
:104F9300D75FC75FBF3F85DD651B757C85DD8E3EB3
:104FA300965E967E969F655C54FB4CFC44FE44FEE5
:104FB30044DD7E1EBF5FC71FBF1EB6FFAE9E961D9C
:104FC3008E3D8E5E969EA71F7DFD54DB551D4CFDC9
:104FD3005D5C9EFFA6FF967E963DA69D9E9DAF3F80
:104FE300865E54FB54FB5D5D8DBB847095979E5D1F
:104FF300A6DEAEFF759C553C657E6DBE75FE96BF05
:10500300A6FF863D6DDD5D9D4D5E4D5F453F4D3F8A
:105013004D3F555F4D5F4D7F55BF55DF65FF7E3F6C
:10502300863F865F7E3F7E3F7E1F8E5FA69FB6FFD5
:10503300BEDFBEDFBEDFBEBFBEDFB6BFA69F9E5FC5
:10504300965E861D7E1E6DFE6E1E661F661E5DDFEE
:10505300559F559F557F4D7F4D7F4D7F4D7F4D9F75
:10506300459F4D9F4D9F4D7F4D9F4D9F4DBF4D9FE5
:105073004D9F4D9F4D9F4D9F4D9F4D9F4D9F4D9FCD
:105083004D9F4D9F4D9F4D7F4D9F4D9F4D9E4D9EDF
:105093004D9F4D9F4D9F4D9F4D9F4DBE4DBE4D9F6F
:1050A3004D9F4DBF4D9E4D9F4DBF4D9F4D9F4D9F5E
:1050B3004DBF4DBF4DBF4DBF4DBF4DBF4DBF4DDF6D
:1050C3004DBF4DBF4D9F4D9F4D9F4D7F4D7F4D7F9D
:1050D3004D9F4D9F4D9F4D9F4D9F4D9F4D9F4D9F6D
:1050E3004DBF4DBF4DBF4D9F4D9F4D9F4D9F4D7F1D
:1050F3004D7F4D7F4D7F4D7F4D7F4D7F4D7F4D7F4D
:105103004D7F4D7F4D7F4D7F4D7F4D7F4D9F4D9FFC
:105113004D7F4D7F4D7F4D7F4D7F4D5E5D9D865E07
:10512300AEFFAEDFB71FAEFF9E9E965D9E7E9E5E78
:10513300AE7EAE7FAE9F96BF65BF4D9F459F459F99
:105143004DBF45BF45BF4DBF559E65BE75FE863FEE
:105153008E5F967F967F9EBF6D7B6D5B865E659D42
:10516300AEDDAEBCB67CBEDDBF1FC73FCF3ECF3F7B
:10517300D75FCF7FCFBF861D54BC54FD4CDD44FEAB
:105183004CFF4CDE653D9EDFA6FE9E9D969E8E5F88
:1051930075BD85DCB71FBEFEC6FEC73EC79F965DC5
:1051A30054BC4CDE453D557D6DBD8E9E8E9E861D49
:1051B3007DBB8E3DAF1FB75FBF7F967D5CDA5D5DC4
:1051C30065BE7E7E865D85BB9578948FC6DAA69E86
:1051D300657B657D6DBD7E3E6D9D967EA6FF96BF0C
:1051E3006D9D759D75FD659D555E4D5E4D5F4D7F56
:1051F300559F559F559F55BF5DDF6E1F7E5F8E7F09
:10520300965E8E3F8E3F863F7E1E7E1F865F8E5E3E
:105213008E7F867F7E1E75DD75DD75FD65DD6E1EF9
:105223007E3D865E867F7E7F6E5F663F5DFF55BEF9
:10523300559F4D9F4D9F4D9F4D9F4D9F4D9F45BFEB
:105243004D9F4D9F4D7F4D7E4D7E4D9E4D9E4D9E60
:105253004D9E4D9E4D9F4DBF4D9F4D9F4DBF4DBF8D
:105263004DBE4D9E4D9F4D9F4D9F4D9F4D7F4D7FFD
:105273004D9F4D9F4D9F4D9F4DBF4DBF45BF4DBF53
:10528300559E559E65FE763F5D9E4D7E4D9F4D9E80
:105293004D9E4D9E4D9E4DBF4DBF4D9E4D9E4D9E71
:1052A3004D9E4D9E4DBF4DBF4D9F4DBF4DBF4DBFFD
:1052B3004DBF4DBF55BF4DBF4DDF4DDF4DDF4DDF03
:1052C3004DDF4DDF4DDF4DBF4DBF4D9F4D9F4D9F7B
:1052D3004D9F4D9F4D9F4D9F4D9F4D9F4D9F4D9F6B
:1052E3004D7F4D7F4D9F4D9F4D9F4D9F4D9F4D9F9B
:1052F3004DBF55BF4DBF4D9E4D7E557E555D6DFED9
:10530300867F865E965E9EDF969F967E9EBF9E7E7E
:105313009E5EA65E9E5F865F65DE4D9E459F459EB3
:10532300459E459E4DBF4DDF559E5DBE6E1F6DFE76
:1053330065BD65BD5DBE5DDE559D4D3C5D5C65DD5A
:10534300F7FFF7FFE7DF9E3C653A5D3C659E75BD61
:105353008E1D967CA6BD8E1E757C657D555D4D1D8F
:105363004CFE54FE5CDB9EBECFBFD75FD75FD73EFC
:10537300CF5EB6FE6D5B5D5D657E75FD867D869E4B
:1053830075FE6DBE659D551B551AAEFFD77EE77E34
:10539300EFFFC75E7DBA75BB861C969F75FE6DBE1B
:1053A300655C8E5DB75FB75FAE9C7C94753A7DDFBD
:1053B300761E65FD6D7C967EAF3F9EDE6D7C6D9D9A
:1053C300659E65BD8E3D9EFF86BF55BD4DBE4DDFBF
:1053D3004DFF4DFF4DDF55DF5DFF661F765F7E3E60
:1053E30075FD75FD7E3F7E3F6E1E6E3F6E3F6E1EEA
:1053F30065FE5D9D65DD6E1E763E767F6E5E6E5F3D
:10540300663F5DDF55BE559E559E4D9F4D9F459F03
:10541300459F459F457E459E459E459E459E4D7DA8
:10542300557D5D9D6DDE75FD6DDD6DFD761D7E1E0D
:1054330075FE75FE65BE65BE5DDE5DDF5DBE5DDE70
:10544300661F663F55BE4D9F4D9F4D9F559F4D9F78
:105453004D9F4D9F4D9F5DFF661F4D9E4D9F4D7F01
:10546300557D6DBD8EBF969F7E1E5DBE559E5DBDF7
:105473006E3E65FE5DBD55BE5D9D761D761D75FD5B
:1054830075FE6DBD65BD765F5E1F4DBE55DF55DF95
:105493004DBF4DDF4DDF4DDF4DDF4DDF4DDF4DDFC9
:1054A3004DDF4DDF4DBF4DBF4DBF4DBF4DBF4D9F79
:1054B3004D9F4D9F4D9F4DBF4D9F4D9F4D9E4D9E6B
:1054C3004D9F4D9F4D9F4DBF4DBF4DBF55DF55DF89
:1054D3005DFF5E1F5E3F663F763F761F7E3F761F12
:1054E3006DFF6DFE65DE6E3F65FE65DD65FE6DFE7F
:1054F300761F661E661E5DDD559D559D65BD75FD5A
:1055030075FD75DD863F7DDD7DDD8E5F8E7F861EBD
:105513007DDC863E865E863E861D967EA6BFA6DF22
:10552300FFDEFFDFF7BFCF9F863E557E455E453DDD
:105533004D1D551D5CDB85DCBF7FBF3FB71FA6DF5D
:105543009EBE967E963D963EA69EB6DEC71FC73E7E
:10555300C73EB75F75DE44FD453F451F4CFD54FB19
:105563009EBEC75FC6FFC71EBEFDE79FF7BFFFBF57
:10557300F7DFE7DFBEFEA65DAE9EBF1EC75EC77E3A
:10558300C75FC6FEC6FE965B861C75DD5D9E4CFE40
:105593006DDCAF3FBF1FA6BF7DDD75DD75DE6DBD65
:1055A3006DBC9EFFA71F7E1C6DFD55BE4DBE4DDF1E
:1055B3004DFF4DFF55DF55DF4DBF55DF5DDF55BE59
:1055C3005DDE661F661F5DFF5DDF55DE55DF55DF60
:1055D30055BE5DBE765F7E7F763F6DFE6DFE5DBE22
:1055E300559E4D9E557E5D9D5D7D5D5C5D5D659DBE
:1055F300659D65BD6DFE75FD6DBC75DC861D8E5D9F
:105603009E9DAEBEB6FFC73FBEFFBEFFBF1FBF1FFF
:10561300BF1FB71FA6BF967F8E7F8E7F7E3F7E5EA6
:1056230086BF765F559E4D7E4D9F4D9F4D9F4D9FEF
:105633004D9F4D9E5DBE7E5F865F65BE559E5D9EA2
:1056430075FE967EA6BFA6BF9E9F7E5F6DBD867FBD
:105653009F1F971F7E5E559C7E5EAEFFB6FFAEDF3B
:10566300AEBFA69F965E96BF663F4DBE4DBE4DBE76
:105673004DBE4DBF4DBF4DBF4DBF4DBF4DBF4DBFC8
:105683004DBF4D9F4D9F4D9F4D9F4D9F4D9F4D9F97
:105693004D9F4D9F4DBF4D9F4D9E4DBF4D9E4DBF49
:1056A3004DBF4DBF4DBF4DBF4DBF55DF55DF55FFFF
:1056B30055FF5E1F5E1F765F863E965FA6BF8E5FB9
:1056C300761E65FE5E1F5E1F5E3F5E3F55FE661FD4
:1056D300661F561F561E5E1E6E1E7E3E9E9FB6FFA3
:1056E300B6DFB6BFB6BFB6DFB6DFAEDF967F7E1ED0
:1056F300861D9E9EAEDFBEDECF1FCF3FC73FAEDF10
:10570300F7BFF79FEF9FD75F963C6D7B553C4D3DB1
:10571300451E44FF54FE755CBF5FD77FDF7FDF7E8E
:10572300D77DD79EC7BF9E9E653B5D5D657E657ECB
:10573300659E6DDE7E1E865E75FD6DBE757E95FD76
:10574300CF5FEFDFF7BEFFDEFFFEFFDFF79FEFBEAA
:10575300EFBEEF9FF79FEFBFF7BFFFDFF7BEF7DFA8
:10576300F7DFF7FFF7BFDF7EC6DDCF3DC79FB6FF8D
:10577300A6FE8E3D85FD8E9F75BD657D6D9D9EDF6D
:10578300B73F9E5E659C6DFE6DFE5DDE5DBF557E23
:105793004D5E555E559F559F4D7F4D9F459F459F40
:1057A3004DBF459F4DBF4DBF4DBF55BF4DBF55BFAE
:1057B3004DDF4E1F4DFE4DDE4DBE459E4DBE4DBED3
:1057C3005D9D7E5F969F9E9FAEDFAEBFAEBFAEBFB9
:1057D300B6BFBEFFC73FC71FC6FED73FDF7FDF9FF2
:1057E300DF9FDF7FD73EDF1FDF3FDF3FDF3FD71E78
:1057F300CEDEC6FFB6BEAE9EA67EA69FA69F8E5EDB
:10580300861D75DD6DDE65DF55BF55BE557E5DBEFC
:10581300661F5DBD6DDE865F9EBF7E1E6DFE867F4D
:10582300969F9EBF965E9E5F9E5F863F7E3F867F6E
:105833007E1D75FC75FD6DFE8E7FAE7EAE7EB67EE3
:10584300B69FB69FAE9F9E5E6DFE5DDF5DDE55DE4D
:105853004DBE4DBE4DBF4DBF4D7F4D9F4D9F4D9F87
:105863004D9F4D7F4D7F4D9F4D9F4D9F4D9F4D9F15
:105873004D9F4DBF4DBF4DBF4DBE4DBE5E1F55DF4E
:105883004D9E4DBF4DBF4DBF4DBF4DBE4D9E559D12
:1058930065FE65FE6DDD7DFDA69EB6DFAE9E9E9F19
:1058A3008E9F6E3F561E55FE561E55FE55FE55FEE7
:1058B30055DE5DDE5DDE761F869F969F9E9FA69ECC
:1058C300A67DA67EAEBEA65D963D863D65DD5DDE0C
:1058D30065DE8E7FAEDFBEFFBEBFB6BFA69E8E7FE8
:1058E300E77FDF3ECEFDDF7FCF1EBEFEA6DE9EBE80
:1058F300969E8E7D8E3D8E1CAEBDBEFEC71FD73ECF
:10590300D73ED75EC77FBF3F655C4D3E4D1E451EEC
:10591300453F44FE759DC77FCF5FCF5FCF3EE79F77
:10592300F7FFF7DFFFDFFFBFFFDEFFDFFFDFF7BFBD
:10593300F79FF77FF77FFFDFFFDFFFDFFFDFFFDF8C
:10594300FFBFFFBFFFDEFFDEFFFFFFFFEFFFB69CE2
:10595300AEFF96BF5D5D54FB7DBBAF1FAEFEA69D44
:105963009E3C961B75BC6D7B8E5DAF3F8E3D6D5A25
:10597300863E6DBD5D5D557E457E459F4D9F4D7E4B
:10598300557D4D7D4D7E4D7D55BE4D9E4DBE4DBECF
:105993004DDF4DFE4DBD4D9D4DBF4DBF4DBE5DBD5C
:1059A30085FDAEBEBEFFCF1FD73EDF3EDF7FDF9F4D
:1059B300E79FE77FE77FE77FEF9FEF7FE75EE77F85
:1059C300E77FDF5FDF7FDF5FDF5FDF3EDF3EDF5FDE
:1059D300D71FC6DEBEDFAE7DAE5DC6FFD75FCF1F6E
:1059E300BE9EB6BEAEBE9E9F969F7E1D865E96BF32
:1059F3009EBF965E8E3E8E5E863D865E865F8E3E43
:105A030075BC65BD6DFE761E7DFD6DFE65FE55BDE7
:105A1300661E5DDD6DFD75DD8E1DB6BEBEBEBEDED2
:105A2300C6FFC6FFC6DFB67EA65EA67FA6BF969F4D
:105A33007E3E6DFD6DDD65DE5DBE559E559E559EBC
:105A43004D7E4D7E4D7E4D7E4D7E4D7E4D7E4D7EFB
:105A53004D7E559E55BE55BE5DDD6E1E763E6DDD9B
:105A630065FE557E4D9E4D9E4D7E557E659D861EE3
:105A7300AEFFAEBE9E7EA6BEA67E9E5E8E1E75DD6C
:105A830065DE559D4D7D4D7D4D7D4D7D4D7D4D7D22
:105A93004D7E4D7D4D7D5DBE65DE5D9D5D9D5DBD38
:105AA3006DDD7DFD75FE6D9D6DDE65DE55DE55FE9E
:105AB3004DDE5DDE6DFE75DE6D9D659D559E559ECD
:105AC300DF3FD6FECEBDDF7FDF9FE77FEF7EE79E22
:105AD300E79EDFDFD7FFC7BF8E5C6DDC75FD75FD0D
:105AE3007E1D7E1C8E3D965D967E8E5E85FD75BC0D
:105AF3006DBC6D9C7DBBB71FCF9FD79FDF5EEF9EB5
:105B0300FFFFFFDEF7BFF7BFFFDFF7BEFFDFFFDFFC
:105B1300FFDFFFDFFFDFF7DFFFDFFFDFFFDFFFDF9A
:105B2300FFDFFFDFFFDEFFBDFFDEF7DFE7DF95DA35
:105B33006D5A6DDD8E7EB6DED75EE7BFE7BFDF9EB3
:105B4300DF5ED73DD77FD77FD75EE79FD73ECF3E78
:105B5300E7FFCF9EBF5EA6FE861E75BE6DBC75BBFE
:105B63009EDDAEBEB6DE965D7DFD761E661E663F8D
:105B73006E3F761F763E6E5E665F665F763E9EBEC6
:105B8300BF1FC6FFD73FDF5FE75EE75EE77FEF9F9D
:105B9300EFBFEF9FEF9FEF9FEF9FEF9FEF9FE79F7A
:105BA300E79FD75EDF5FDF7FDF7FDF7FE77FE79FF3
:105BB300DF5ED75FD75ED75EDF7FEFBFF7DFF7DF4D
:105BC300F7BFEF9FE77FDF7FD79FCF7FCF5EC73ED4
:105BD300BEFDBF1EB6FEAEFE9EBD9EBDA6DDAEDD06
:105BE300AEDCA6DD96BD9EFEA6DE967D967D9EBEB0
:105BF300AF1EB71DB6FDBF1DCF3ED77EDF7EDF7E56
:105C0300DF5ED75ED75FCF5ECF3ECF3ED73ED73E78
:105C1300CF1DC71EBF1EB73EAF1EA6FEA6DE9EBD8E
:105C23009EBD969D969D969D969D969D969D96BD91
:105C3300969D96BD9EBEAEFEB71EC73FBF1EBEFE5F
:105C4300B6DEA69D9E9D969D969D9EBEB6FECF5F9B
:105C5300DF5FDF7ECF5FC73EC71EBEFEAEBE9E7D4B
:105C63008E7D969E967E967D967E969E969E969E1B
:105C7300969E96BE96BE8E9D969D969E969D9EDE04
:105C8300A6FEAEFE9EBE96BE8EDE96DE9EBEA6DE51
:105C9300A6BD9EBD9E9D969E969E8E9E8EBE8E9EFC
:105CA300DF1ED6FECEBDDF7FDFDFE7BFEF9EEF7ED9
:105CB300EF5EEF7EDF7FCF9F9E9C6DDB65DC5DFD3E
:105CC30055FE5E1E65DD6DBCAEDEDF7FD79FCF9ECA
:105CD300CF9EC79FC77FA67C7DFB85FBAE9CEFDF76
:105CE300FFDEFFBEF7DFF7DFF7BFF7BFF7DFF7DF53
:105CF300FFFFFFFFFFFFF7DFF7BEF7BEF7DFF7DFBB
:105D0300FFDFFFDFFFDFFFDEF7BEF7DFEFDFCF5E93
:105D1300AEBD9E9EBEDDF7DFFFFFFFDEE73CD6BBD9
:105D2300E75EFFFFFFFFFFDFFFDFFFDFFFDFF7BE02
:105D3300F7BEF7DEEFBEE79FD77FBEFEB67DBEBCE4
:105D4300E7DFEFBFEFBFDF9FCF5FBF3F967D75DC20
:105D5300759C8DFD863E6E1D561D5E1E7E7F9E9F2D
:105D6300A6BF9EBFA6BFA6BFAEDFBF1FC71FC73F4D
:105D7300CF3FCF5FCF5FCF3FCF3FCF3FD75FD75F20
:105D8300D75FC6DDBEBDC6DDD73FDF5FDF7FDF7E0A
:105D9300DF3DE77EF7DFFFFFFFDFFFDEFFDEFFFE16
:105DA300FFDEFFDFFFDFF7DFEF9EE77ED75EC73E55
:105DB300AEBD9E5C8E3D861D7DFD75FD7E1CA6BE23
:105DC300BF5FB75F7DFC659C75FD9E5CBEFDAE5CF1
:105DD300BEDDDFBFDF7FDF7FDF7FDF5FE75FE75EA4
:105DE300DF3ED73EC6BDBE9DB6BDBEDDC6FEC6DE2A
:105DF300B69EA69E969F86BF767F65FE65DE65FE90
:105E03005DFE5DDE5DFE65FE5DFE5DFE5DFE65FEC7
:105E130065FE65FE65FE767F86BF869F869F7E5EF6
:105E23007E7E763E661E661E6E3E6E1E7E5E8EBF56
:105E33008E9E96BF8E5E8E5E8E7E969F7E1D6DFDC0
:105E43006DFD661D661E661E661E663E663E663EEA
:105E5300663E6E1D6E1D6E1D6E1D761D761D763E95
:105E63007E1D865E7E7F6E3E663D6DFD8E3DAEBFC2
:105E7300AEDFA6BE865D6E1D661D65FD65FD6DDD2F
:105E8300EF9FEF9FDF7FC71EAE9CA69DAEDECF7F49
:105E9300E7BFEF9EEF9FE79FC71E8E3C6D9C5D5C47
:105EA300557E4D7E557E4D1D8E1EDF7FDF7FDF7E4F
:105EB300E77EDF7EDFBFAEBD551A761CB6FDE7BFBA
:105EC300EFBFF7BEFFFFF7DFF7DFF7DFF7DFF7DF40
:105ED300F7DFF7DFF7DFF7DFF7BFF7BFF7DFF7DF4F
:105EE300F7DFF7DFF7DFF7DFF7BFF7BEF7BEF7BE82
:105EF300F7BFF7BFF7DFF7DFFFDFFFBFF7BFF7BF7F
:105F0300F7BFF7DFFFDFF7BFF79FF7BFFFDFF7BF8E
:105F1300F7BEF7BEEF7EEF7EEF9FEFBFE77EEF9F0B
:105F2300F7BFF7BEEFBEEFBFEFBFE79FDF7FD75FE0
:105F3300BEBDBEFEBF7F7E3D55BC4DDF5DDF6DFF49
:105F430065FF5DFF5DDE5DFE5DDD6DFD861E965FBB
:105F5300965E963D963D9E5E9E7EA6BFA6BFB6BE4E
:105F6300BEDEBEDEB69EC6FFD73FD73FD73EDF3E7F
:105F7300EFBFF7FFFFDFFFBEFFDEFFDEFFFFF7FF31
:105F8300FFFFFFDFFFDFF7BFEF9FEF9FF79EF7BE38
:105F9300E77ED73ECF3ED77FCF7FAE9DB67CDF7FF8
:105FA300DF3ECEFEB65CB69DCF5FEFDFEFDFDF3DBA
:105FB300E77EEFBFDF3ED71FDF1FD73EE79FEFBF71
:105FC300E77FDF3ED73ED75FCF1DD73ED77FBF1FCB
:105FD3009EBF7E3E5DBE55BE559E559D55BE55DF4B
:105FE30055BF4DBF4DBF55DF4DBE4DBE4D9E4DBE42
:105FF3004DBE4DBE55BE4DBE55DE55DE55DE5DDF95
:1060030055DF4DBE4D9E55BF55BE55BE55BE55BE03
:1060130055BE55BD55BE55BE55BE55BE55BE4DBEEE
:106023004DDE55DE55DE55DE55DE55DE55DE55DEDD
:1060330055DE55DE4DDE55DE55DE55DE55DE55DECD
:106043005DDE5DDE55DE4DDE55DE5DBE6E1E863FDA
:10605300863E7E5F6E3F5DFE55DE55DE55DE55DEC8
:10606300F7DEF7FFE7DFAE9D859B8DDDAE5FB69E66
:10607300C6FEE79FEFBFEF9EEFDFEFFFDFBFCF3E31
:10608300C73FBF1FB6FFAEDEA6BEA6BEA6BEC71FD6
:10609300DF5FDF3DD77EBF5FA67DC71EE7DFE79FDC
:1060A300EF7FE75EF7DFF7FFF7FFFFFFF7FFF7DFAE
:1060B300E77EEF7FEF9FEF9EF7BFF7DFF7DFF7FF97
:1060C300F7DFF7BFF7BFF7BFF7BFF7BFF7DFFFDFB5
:1060D300FFDEFFDEFFDFF7FFFFDEFFBEF7DFF7DFE9
:1060E300FFFFFFDEF79EF7BFF7DFF7DFF7DFF7DF2F
:1060F300F7BFEFBFDF5FD71EDF3EE75FE77FEF9FAF
:10610300F7BFEF9FE77FE77EEF9FEF9FEFBFF7DFDD
:10611300F7DFEFBEEFDFBF3F6DBC4D9E4DDF4DDFC1
:106123004DBF4DBF45DF4DFF55FE6DFE8E5F965F44
:10613300967E965E965E965E963E8E3D963EA69EB5
:10614300B6BFB6DFBEFFC6FFC71FCF1ED73EEFBF2A
:10615300F7FFFFDEFFBEFFDEFFDFFFDFFFDFFFDF57
:10616300FFDFFFDFFFBFF79FEF9FEFBFF79FF79EB5
:10617300EF9EEF9EEFBFE79EE77FE7BFE79EEF9EB1
:10618300F79EEF7FEFBFF7DFFFBEF7DEF7DEF7DF48
:10619300FFDFF7DFE79FD75FCF1FC6FEDF7FE79FF6
:1061A300E79FE77EE79FE7BFD75FB6BE8DFC6DDD58
:1061B300661F4DBE4D9E4D9E559E5DFF5E1F4DBE9F
:1061C30055BF4DBF4D9E4D9E4D9F4DBF4DBF4DBFC6
:1061D3004DBF4DDF55DF4D9F4D9F4D9F4D9F4D9FB4
:1061E3004D7F4D7F4D9F4D9F4D9F4D9E4DBE4DBE4F
:1061F3004DBF4DDF4DBF4DBF4DBF4DBF45BF4DBF24
:106203004DBF4DBF4DBF4DBF4DBF4DBF4DBF4DBF2B
:106213004DBF4DDF4DDF4DDF4DDF4DDF4DBF4DBF7B
:106223004DDF45DF4DDF4DBF4DBF4DBF4DBE4DDF94
:106233004DDE4DFE55FE55FE561F561F55FF4DDFD5
:10624300F7BEEFDEE7DFBEFFA69FA67FAE5FAE3EE3
:10625300AE3EBE7ECEFECEFDD73DE7DFE7DFE79E57
:10626300E79EE79EDF9FDFDFC79F85DC961DBEBFEE
:10627300C6FFC6DEBEBEB6BDE79FF7DFF7BFEF7E44
:10628300E77EE77ED75FD73FDF3ED73FDF5FDF7F26
:10629300DF7FE75EE75FEF5EEF7FEFBFEFDFEFDF0D
:1062A300F7DFF7BFEF7EEF9EEF9EF7DFFFFFFFFF06
:1062B300FFFFF7DFF7BFFFDEFFDEFFDEFFDFFFFFDE
:1062C300FFFEFFDEF7DEFFDEFFFFFFDFF7DFF7DFB7
:1062D300F79EEF9FE77FDF5EE75EE75FEF9FEF9F4E
:1062E300F7BFF7BFEF7EEF7FEFBFEFBFF7DFF7BF7C
:1062F300F7BEF7BEEF9EE7DFBF1E969D869D7E9D90
:10630300767D767D7E9D7E9D96DEAF1FB6FEBEFEBC
:10631300BF3EBF3EC73EC73ECF3EC71EC6FDC6FDFE
:10632300CF1ECF3ED73ED73EDF5EE79EF7DFF7DFD8
:10633300F7DFFFDFFFDFF7DFF7DFF7FFFFDFFFDF6A
:10634300FFDFFFBFFFBFF7BFF7BFF7BFF79FF7BF82
:10635300F7BFEFBFEFBFEFBFEFBFEFBFEFDFF7DF7A
:10636300F7BEF7DFF7DFF7DEFFBEFFBEFFDEFFBDE1
:10637300FFBEFFBEF7BEEFBFDF7ED75EDF7EDF9FD0
:10638300DF7FD75ECF5EC73EA6BD9EBE865C763DF1
:106393006E5D6E7E6E5D765D767D767D765D765D19
:1063A300765D765D6E5D6E5D6E5E6E3E6E5E6E3EBE
:1063B3006E3E6E3E6E3E6E3E6E1E6E1E6E1E6E1EFA
:1063C3006E1E6E1E661E663E663E663E663E663EFA
:1063D300663E663E663E661E6E1E661E661E661E32
:1063E30065FE65FE65FE65FE65FE5DFE5DFE5DFEAA
:1063F3005DFE5DFE5DDE5DFE5DDE5DDE5DDE5DDE62
:106403005DDE55FE55DE5DDE55DE55DE55FF55FF7F
:1064130055FF55FF55FE5DFE5DDE5DFE55DF55DF25
:10642300DF5EE77FE7BFCF3EB6BDAE9E9E7E9E5E3C
:10643300A65EA65EAE7EAE5EB69EDF9FE7BFE7BFFB
:10644300E7BFE7BFE7BFE79FD7BFAE7CBEBDC6FFD1
:10645300BEBEB69FAE5EB67DD73EEFDFE77FEF9E53
:10646300EF9EE7DFCF3F9DFD961E9E5FA67FA67D35
:10647300C71EE79FE77FEF7FEF9FDF3EC6BDCEFFDF
:10648300CEFFDF3FE79EE7BEEFBEF7BEF7BEFFDE00
:10649300FFDEF7DFFFDFFFDFFFDFFFDFFFFFFFFFD2
:1064A300F7DFF7BEF7DEFFDFFFDFFFDFFFBFF7BF7B
:1064B300F7DFF7DFEFBFEF7EEF7EEF9FE77EEF9F24
:1064C300E77FE75EDF3EDF3FDF5FDF5FE77FE75EBC
:1064D300E79EE77EE77EDF7FDF7FBEDDAE9CA67DA6
:1064E300863B865C7DFC861C8E5D967D9E5CA69CB1
:1064F300B6BDBEDDC6FDCEFDCEFDD71ED75ED75ED3
:10650300CEDDC6DDD73EE77EEF9FEFBFEFBFF7BF20
:10651300F7BFF7BFF7BFF7BFF7BFFFBFFFDFFFDF70
:10652300F7BFF79FEF9FF79FF79EF79EF79EF79EA4
:10653300EF9EEF7EEF7FEF9FEF9FEF9FEF9FE77F52
:10654300EF7FEF9FF79FF79FF79FEFBFEFBFEFBF80
:10655300F7BEF7BFF7BFEF7FDF1DDF3EDF3ED73F5D
:10656300C73F965D7DFC6DFC5DBC5DDD5DBD5DDDA6
:106573005DBD55BD55DD55DD55BD55BD55BD55DD20
:1065830055DD55DD55DD5DBD5DBD5DBD5DBD5DBDF0
:106593005DBD5DBD5DBD55BE55BD55BD5DBD55BD47
:1065A30055BD55BD55BD55BE55BD55BD559D5D9D8F
:1065B3005D9D5D9D55BD55BE55BE559E559E559ED3
:1065C30055BE55BE559E559E559E55BE55BE55BE90
:1065D30055BE55BE55DE55BE559E559E55BE559E60
:1065E300559E4D9E4D9E4D9E4D9E4D9E4D9E4D9E48
:1065F3004D9E4D9E4D9E4D9E4DBF4DBF4DBE4DBFBD
:10660300BEBECEFED6FEE75EEFBFE7BFE7BFE79FA6
:10661300E79FE77FDF5FDF5FCF3FA69D8E3C8E9DC9
:106623008EBD8EDD9EDDB6FDBF1ECF5FD77FD75EED
:10663300C6FEB69DB69EB69EB6BCCF3EDF7FDF5E7E
:10664300DF7ED77ED77F9E1D7DDE85DE8DFD95DBCC
:10665300A63BDF9FDF9FE7BFE7BFD75FAE1EADFE61
:10666300AE1EB63DDF5FEFDFEFDFF7DFEF7EF79DB7
:10667300F7BEF79EFFDFFFFFFFDFF7DFF7BFF7BFD1
:10668300F7BFF7DFF7BFFFBFFFBFFFBFFFBEFFBF10
:10669300FFDFF7DFF7BFEFBFE79FE77FDF5FDF7F57
:1066A300DF5FD71FCEFFC6FFC6DFC6FFC6DECEFE47
:1066B300D71EDF5EDF5FDF3FD71ED73ECF3FCF3F23
:1066C300BF1FAEDF8E7F7E5F765F7E5F8E9F9EDF16
:1066D300AEFFB71FC71FC71FC71FCF3FCF5FCF5F18
:1066E300CF3FC71FCF1FCF3FD75FDF9FDF9FDF7F27
:1066F300DF7FE77FE77FEF9FF7BFF7BFF7DFF7DFC7
:10670300F7BFEF9FEF7FEF7FEF9FEF9FEFBFEF9F0E
:10671300EF9FEF9FEF7FE75EDF3ECF1FBEDFBE9EA3
:10672300BEBEBEBEC6BEC6DFC6BEBEDEBEFEC6FFA4
:10673300CF3FCF3FCF3FC71FC6DFBEBFB6BF9E7F92
:106743007E1E5DDD4DDE45FF4DDF4DDF4DDF45DF59
:1067530045DF45DF45DF4DDF4DDF4DDF4DDF4DDFEE
:106763004DDF4DDF4DDF4DDF4DDF4DDF4DDF4DDFC6
:106773004DDF4DDF4DBF45BF45BF45BF45DF45DF5E
:1067830045DF45DF4DBF4D9F4D9F4D9F4D9F4D9F16
:106793004DBF4DBF4DBF4DBF4D9E55BE4D9E4DBFD1
:1067A3004DBF4DBF4D9F4D9F4D9F4D9F4DBF45BF0E
:1067B300459F4DDF55FF4D9E4DBE4DBF4D9F4D9F98
:1067C3004D9F4D9F4D9F4D9F4D9F4D9F4D9F4D9F66
:1067D3004D9F4D9F4D9F4D9F4D9F4D9F4D9F4D9F56
:1067E300BEDFCF1FD6FEDF3EEFBFEF9EEF9EEFBEB5
:1067F300EFBEEFBFE7BFE7BFDFBF861E553C55BE09
:106803004DDE55DE5DBD7E1E9E5ECEFFEFDFEFBF2C
:10681300E79EDFBFDFBFDFBFCF7FA65CBEBEC6DEA6
:10682300C6DDC6DDBE9DC71FD77FCF1ECF1ECF1EC1
:10683300C71EAE7D9E5DA65DAE9EAE9EB69EBEDEBF
:10684300BEBEBEBDD73EDF5EDF5EE79FEF9FEF9E1E
:10685300F7BEF79EFFDEFFDEFFDFFFDFF7BFF79E2A
:10686300FFBEFFDFF7DFFFDFF7BEF7BEFFBEFFDED2
:10687300FFDFF7BFE77FD71ED6FDCEDDC6DEC6BE80
:10688300C6DEC6DFBEBFB69FAE9FB69FB6BEBEDF37
:10689300CF3FD73FD73FD6FEDF1EDF5EE77EDF5F0A
:1068A300D73FB6DF8E3D761E6E3F765F763E8E5EB9
:1068B3009E7EA69EAEBEB6DEBEDEBEDEBEFFBEDEE4
:1068C300B6DEB6BEB69DAE7DB6BEBEDEB6BDA65DB9
:1068D300A65DA65DA65DAE9EB6DEBEDFC73FCF3E1C
:1068E300C71FC6FECF1FCF1FD73FD75FD77FDF7F1F
:1068F300DF5FDF5EDF5FD73ECF1EC71FC6FFC6FF6A
:10690300BEDEBEBEBEBEB67DB67EAE3D9DFC95FD73
:1069130085FD861D761E761E6E1E661F65FF55DE7F
:106923004DDF4DFF45FF45DF4DDE55DE55FE55DEA0
:1069330055FE55DE55DE4DFE4DFE4DFE4DFF4DFF22
:106943004DFF4DFF45FF4DDF4DDF4DDF4DDF4DDF8C
:106953004DDF4DDF4DDF55BE55BE4DDE4DDF4DDF07
:106963004DDF4DDF4DBF4DBF4DBF4DDF4DDF45DF2C
:1069730045DF45DF4DBE55BE65FE7EDF65FD559D9A
:1069830055BE4DBE561F55DF4DDF4DDF4DDF4DDF8D
:106993004DDF4DDF4DBF4DDF4DBF4DBF4DBF4DBF34
:1069A3004DBF4D9F4D9F4D9F4D9F4D9F4D9F4D9F64
:1069B3004DBF4DBF4DBF4DBF4DBF4DBF4DBF4DBF74
:1069C300AE5DBEBEAE3CC6DDEFFFF7FFF7DFF7DF20
:1069D300EFFFEFFFEFDFE7DFE7FF8EBE557D4DBE35
:1069E30045BE4DDF55BE5DBD7DFD95FCD79FE7BF21
:1069F300E7BEE7BEE7BEE7BEDFDFBEDEB67EC6FFAD
:106A0300CF5FD77FC6FFD75FF7DEF7BEF7BEEF9E38
:106A1300E7BFB6DE7D9C7DBE85BD859BAE9DDFFF5A
:106A2300DFBFE7BFE7BFBE9CB65CCF3FE7BFF7FF63
:106A3300F7DFFFDFF7DEEFBEE79FE79FE79FF7DFB5
:106A4300F7BFF79FDF7FDF9FEFBFF7FFF7DFF7DFCB
:106A5300EFBFEFBFE77FDF3ECEFEC6DEBEBEBEBEEC
:106A6300BEDFB69FAE9FAE7FA67FA67FB6BFBF1F1A
:106A7300C71FC71FCEFFCEFEDF3EE79FEFBFE77FF7
:106A8300D75FBEDFA69E8E5E8E7F7E1D7E1C8E3CF4
:106A93009E7EAEBEB6DFBEFFC6FFC6FFC71FC71FC3
:106AA300C6FFC6FFC71FC6FFC71FC71FBEDFAEDFB8
:106AB300AEDFA69E965E7DDD75BD6DBD75BC7DDCCE
:106AC30085FD85FD8E1E963D9E3EA67EA67EAE7DF1
:106AD300B69DC6FDC6FDC6FEBF1FC6FFCEFED73F91
:106AE300CF1FBEDEC71FBF1FBF1FAEFF9EBF865F88
:106AF3006E1E5DDE55FF4DFF4DFF4DFF45DF4DFF24
:106B03004DDF55DE5DBE5DBD5DDE5DFE661E663F2F
:106B13006E3E6E3F6E5F6E3E763E763E763E761EF0
:106B2300761E761E763E763E763E763E763E7E5EDA
:106B33007E7F7E9F869F8E7F867F6E5F5E1E561E44
:106B430055FF55DF55DE55FE5E1E5E3F55FE4DFF7C
:106B53004DFF4DFF4DDE5DFE6E5F7E7F765E661EF2
:106B630055DE55FF5E3F665F55DE55DE4DDE4DDE7D
:106B73004DDE4DBF4DBF4DBF4DBF4DBF4DBF4DBF93
:106B83004DBF4DBF4DBF4DBF4DBF4DBF4DBF4DBFA2
:106B93004DBF4DBF4DBF4DBF4DBF4DBF4DBF4DBF92
:106BA300BEDDBEBDB69CB6BDB6DDAEDDB6FEB6FE81
:106BB300B71EB71EB6FEAEDEB71E96BD865C7E3D23
:106BC300763D763E765D765D761C7E3CB73FC77E2E
:106BD300CF5ECF3ED75ED75ED79EBEDEAE3DB65DFF
:106BE300BE9DC6DDC6DECF1FDFBFEFBFEF9FEF7ECB
:106BF300E77FCF3F8DDB7DFD7DDD8DDC95FBCF3EDC
:106C0300DF7FDF5EDF7FBF1EA61BA63CAE3BC6DD7C
:106C1300E79FEF9FE7BFCF1EAE3DAE5DAE5CD77F74
:106C2300DFBFDF9FBEBEB65DB67CD75EE7BFDF9F2B
:106C3300C6BDC69CDF1EEFDFDF7FBEBEBEDFB6DF95
:106C4300B6BFAE9FAE7FA65F9E5FA67FA65EA67E03
:106C5300AE7EB69EB69EC6BED73FE79FDF7FD73ECA
:106C6300BEBEAE9EAEBFA69FA6BFA6DFAEFFB71F3A
:106C7300BF3FC73FCF3FCF3FD73FD75FCF3FCF3F89
:106C8300CF1FCF3FCF3FCF5FCF3FC71FC6FFBEDE74
:106C9300B6BEA69E969E867F763F6E1E6E1E6DFEC8
:106CA3006DFE761F761F761F7E3F7E1E8E1E9E5EB6
:106CB300B6FFC73FC73FAEBE9E5D8E3D8E5E8E7FE5
:106CC300865F75FE65DD661E6E3F661E5DFE55DEE4
:106CD30055FF4DDF4DDF55DE5DDE6DFE6E1E6E3FF3
:106CE300765E7E5E8E9E9EBE9EDFA6FFAF1FAF1FAB
:106CF300AF1FB71FB71FB71FB73FB71FB71FAEFFF2
:106D0300AEFFAEFFAEFFAEFFAEFFAEFFA6FFA6FF28
:106D1300A6DFA6DF9EBF969F8E9F765F5E1E4DFE0B
:106D23004DFF4DDF55BE661E663F5DFE55FF55DFC9
:106D33004DDF4DDF45FF4DDF55BE5DDE5DFF55FF8A
:106D430045DF4DDF4DDE4DDE4DDE4DDF4DDF4DDFEB
:106D53004DDF4DBF4DBF4DBF4DBF55BF55BF55BF98
:106D63004DBF4DBE4DBE4DBE4DDF4DDF4DDF4DDF43
:106D73004DDF4DDF4DDF4DDF4DDF4DDF4DDF4DDFB0
:106D8300EFDFEFDEEFFFBF1E5D1B4D1B4D3B4D3BAA
:106D93004D3C4D5C4D5C4D5C5D9C8E7DD7DFE7BF0C
:106DA300E7BFDFDFD7DFDFBFE7DFCFDF867C5DDB7A
:106DB3006DDD963EAEBEAE7D9E3CBEDDE77FEF7ED3
:106DC300EF9EE79FE79FE7BFCF3EBEBEBEBFC6BFF6
:106DD300BEBEB69CCF5ED79FD77ED75ED77EAEBDF5
:106DE3008DDB85FD7DBD969EC77FD73DD71DC71E15
:106DF3009E5D85FC865E8DFDC6DED71EC73EAEFE5C
:106E03008E1B95FC9E1DC71ECEFDC6DDA63C9E3D7A
:106E1300AE9EC6FDC6FDBEBDAE9D9E5E8E1E8E3E63
:106E2300963E8E3F963E961E95FD8DDC85DD861E35
:106E330085FE8DFD8DFD961E9E3EA67EAE7EA65DD5
:106E43009E7E8E5D8E9E869E869E8E9E967E9E9E48
:106E5300AEBEBEFEC71FC71ECF1FCF1FCF3FCF1F64
:106E6300D71ED73ECF1FCF1ECF1EC6FEC6FEB6DE31
:106E7300AE9EA69D965D8E3D867E867E7E5F763F28
:106E83006E3F663F665F665F665F663E7E1E967F09
:106E9300967F863E863E7E1D75FD763E7E3E7E3F18
:106EA3007E1F6E1E661E661E661E6E1E6E3F6E3E45
:106EB3006E3E763E863E967FA69FAEBEA6FFA71F7A
:106EC300AF1FBF1FBEFFBEFFBF1FB71EB71EBF1F33
:106ED300BF1FBF1EBEFEBEFEB71FB71FB6FFAEDF8E
:106EE300AEDFA6BF9EDF9EBF969E8E7E865E7E5ED3
:106EF300765E763E6E3E5E1F55FE55FE55DE55DED2
:106F030055BE5DFE65FE6E1D767F6E5F661F663F36
:106F130055FE55DF4DFF4DFF4DFF4DFF4DDF55FF37
:106F23005DFF5DFE5E1E5E1E5E1F561F561F4E1FDB
:106F33004DFF4DDF4DDF4DDF4DDF4DBF4DBF4DBF2E
:106F43004DBF4DBF4DBF4DBF4DBF4DBF4DBF4DBFDE
:106F53004DDF4DDF4DDF4DDF4DDF4DDF4DDF4DDFCE
:106F6300EFBFEFBEEFDFC73E757A555B4D7C4D7CBF
:106F73004D5D4D5D4D5C5D9D65DE965DD7BFF7BF95
:106F8300F79EF7BEEFBFEFBFEFBEE7FFA71E6E1D75
:106F93006E1E7E3F863E865F8E3FA65EDF7FF7DFF7
:106FA300F7BFF7BFF7BFF7DFD75FA63C965E865FF5
:106FB3008E7F965EB6DEE7DFEFBEEF9DEFBFCF7F3E
:106FC30085FC75DE6D9E755CBEFFEF9FE79EDFDF80
:106FD3009EBD551A557C557B969DD7FFDFBFD79F26
:106FE300961D7DDE7DFEB73FDFDFD79FA65C7D9BD1
:106FF3008E1CBF5FD7BFAEDD85DB8E3D863D863EF3
:10700300969F9E7FA69FB6DFAE9F9E3D961D8E1ECA
:10701300861E861E85FE8E1F8DFF8E1E963EA69EA5
:1070230096FF661C55FC561D561D561D5DFD763D8F
:107033009E9EAEDFAEDFB6BEBEDFB69EB6BEC6FF59
:10704300CF1FD75FD77FD73FD75FD75FDF7FDF7F85
:10705300D73FCF5FCF5FBF1FB6DFA67E8E5E7E3E7C
:10706300761E6E1E661E661E65FD6DFD863D969F31
:107073008E3E8E1D8E1D9E7EA6BFA6DFA6BEAE9E35
:10708300AEBEA6DE9EFFA71FAF1FB71EB71EB71F5C
:10709300AF1FB71FB71FBEFFBEDFB6FFB6FEBF1ED3
:1070A300C6FEC6DEBEDFAEDFAEDFAEBFA6BFA6DF67
:1070B300A6BFA6DFA6BF9EBF9EDF96DF96BF8E7FCD
:1070C300865F867F763E65FD5DFD55DD55FE55DEAB
:1070D3004DFE4DFE4DFE55DE55FE55FE5DFD6E7EAD
:1070E3007EBE86DE769E663E661E5DFE55DE5E1FB6
:1070F300561F55FF55FF561F4E1F4E1F561F561F37
:107103005E1E5E1F5E3F5E3F5E3F5E3F563F561E06
:1071130055FE4DDF4DDF4DDF4DDF4DDF4DDF4DDFE5
:107123004DDF4DDF4DDF4DDF4DDF4DDF4DDF4DDFFC
:107133004DDF4DDF4DDF4DDF4DDF4DDF4DDF4DDFEC
:10714300FFFFFFDEF7FFC7BF6DFD55BD4DBE4D9E73
:107153004D7E559E557D5DBE65BD85FCCF9FEFFF82
:10716300F7BFF7DFEFDFE7DFEFDFE7FFC79F8E5DF7
:10717300865D863D861D863E761D7DDBAEFDCF9EFC
:10718300CF9ECF7ECF7ECF7EC75E8E1A7DDA7DDC2B
:107193007DFC85DB8E1BBF5ECF7ED77FCF5FBF5F5E
:1071A3009E9D85FB861C7DFCA6BEB73EA6DD9EFE8E
:1071B30096BE8DFC863C865D8E7D9EBE9E9E9E9E6B
:1071C30096BEA75FBF3FB71E9E7C967DA6BEC75FD8
:1071D300D75ECF1CAEBBAE9BB71DBF7FAF1E965E07
:1071E300967F961E9E1EAE7EBEFFBEDFB6BEAEBEB1
:1071F300963D85FE7DDD85FE8E3E8E3F965F9EBF6E
:1072030096DF765F661E663F665F665F663F6E3F2C
:107213007E3E8E7F969F9E9EA69EAEBEAEDFAEBE88
:10722300AE9EB69EB6BEBEFFC71FC6FEC6DECEDE90
:10723300CEFFC6DEBEBEB6BFB6DFAE9F9EDF8E9F5D
:10724300865E867F867F867F8E9F969EA6DFA6DFDD
:10725300AEFFAEFFB71FBF3FC73FC73FC73FCF1FFD
:10726300C73FBF3FB73FBF1FBEFFAF1EAF1EAEFE40
:10727300AEFEA6DEA6BEAEBEA6DFAEDFAE9DC6DD0B
:10728300E79FCF1EA69E969F8E7F8E9F867F7E5FF3
:107293007E5F765F6E1F661E5E3E663E663F665F7E
:1072A300665F5E3F561E4E1F4E1F4E1F4E1F4E1FE4
:1072B3004E1F4E1F4DFF4DFE563F5E5F5E5E667E68
:1072C300665E661D55FD4DDE4DDE4DDE4DFF4DFF09
:1072D3004DFF4DFF4DFF4DFF4DFF4DFF4DFF4DFE4C
:1072E3004DFE4DFF4DFF4DFE4DFE4DFE55FE55FE31
:1072F30055FE4DFF4DFF4DFF4DFF4DDF4DDF4DDF84
:107303004DDF4DDF4DDF4DDF4DDF4DDF4DDF4DDF1A
:107313004DDF4DDF4DDF4DDF4DDF4DDF4DDF4DDF0A
